:020000040800F2
:10000000E85B0020E9010008B54E0008713A0008DD
:10001000E9460008090A0008C95F0008000000005E
:100020000000000000000000000000005101000876
:10003000050B00080000000095010008915700081A
:10004000030200080302000803020008030200087C
:10005000030200080302000803020008030200086C
:10006000030200080302000803020008030200085C
:1000700003020008A90A0008B90A0008C90A000812
:100080000302000803020008E10700080302000859
:10009000030200080302000803020008030200082C
:1000A000030200080302000803020008030200081C
:1000B00045580008615800080302000803020008C0
:1000C00003020008030200080302000803020008FC
:1000D00003020008255F000803020008B95F00085A
:1000E00003020008030200080302000803020008DC
:1000F00003020008030200080302000803020008CC
:1001000003020008030200080302000803020008BB
:1001100003020008030200080302000803020008AB
:10012000030200080302000803020008030200089B
:10013000DFF810D000F008FB00480047256A0008EF
:10014000AFF30080E85B002080F308887047000070
:10015000224B19680868B0E8F00F80F30988BFF3F4
:100160006F8F4FF0000080F311884EF00D0E704736
:100170000000000006480068006880F3088862B646
:1001800061B6BFF34F8FBFF36F8F00DF00BF00BFBB
:1001900008ED00E0EFF30980BFF36F8F0F4B1A6893
:1001A00020E9F00F106008B54FF0500080F311887F
:1001B000BFF34F8FBFF36F8F07F066FC4FF0000067
:1001C00080F31188BDE8084019680868B0E8F00FAE
:1001D00080F30988BFF36F8F704700BFA805002028
:1001E000EFF3058070470000064880470648004747
:1001F000FEE7FEE7FEE7FEE7FEE7FEE7FEE7FEE7D7
:10020000FEE7FEE74358000831010008202A04DB1E
:10021000203A21FA02F00021704721FA02F3D0407F
:10022000C2F12002914008431946704740EA010399
:100230009B0703D009E008C9121F08C0042AFAD29C
:1002400003E011F8013B00F8013B521EF9D2704760
:10025000D2B201E000F8012B491EFBD27047002208
:10026000F6E710B513460A4604461946FFF7F0FFB5
:10027000204610BD421C10F8011B0029FBD1801A3A
:100280007047F0B480EA0102D40F4200B2EB410F94
:1002900002D20246084611464A0042D0C30DDDB2E2
:1002A000C1F3C752AD1A202D35DAC1F3160141F45E
:1002B000000204B15242C5F1200602FA06F12A41B9
:1002C0001044B3EBD05F23D0C4B1012DA0EBC350D9
:1002D00009DCF0BC4FF0004202EAC352DBB200F589
:1002E000000000F0A6B9400000F1807000EBC350A0
:1002F000A0F1807040EAD170490009E0490841EA64
:10030000C071A0EBC35000F50000400800EBC350E3
:10031000F0BC00F085B96142012202EB4101001BF3
:10032000F6E7F0BC704781F00041AAE780F000409A
:10033000A7E780EA010210B502F00043400022D096
:100340004A001FD0010E01EB1261C0F35600C2F348
:10035000560240F4000042F40002A0FB0220000418
:100360007F39140400D0401C50EA124001D44000F0
:10037000491EC2B20C0604EBD010401C4008802A73
:1003800002D003E0002010BD20F00100002900DAB7
:100390000020184310BD30B480EA010202F000458D
:1003A00030F0004221F0004013D090B1C30DD40DC5
:1003B000C2F31601C0F31600E41A41F4000140F440
:1003C00000027D34914201D3641C00E04900002CFE
:1003D00002DA30BC002070474FF400000023914245
:1003E00001D3891A034340084FEA4101F7D151B1C3
:1003F000914202D14FF0004105E002D24FF00101DD
:1004000001E06FF0010103EBC450284430BC00F060
:1004100007B92DE9FE4F81EA030404F0004421F0FE
:10042000004100944FF0000B23F0004350EA010418
:100430005ED052EA03045BD0C3F30A54C1F30A55F9
:100440002C44A4F2F3340194A0FB0254C1F3130131
:1004500041F48011C3F3130343F4801301FB0244FE
:1004600000FB034E840A970A44EA815447EA835703
:10047000A4FB076802958D0A05FB07854FEA932CBC
:1004800004FB0C542705029D4FEA065847EA16372D
:10049000B5EB08056EEB070C870E920E47EA811745
:1004A00042EA8312A7FB0201B6EB0B0164EB0004E6
:1004B0002B0D43EA0C335E1844EB1C50DA465146D0
:1004C000E7FB0201C5F313044FEA0B3343EA14536D
:1004D0004FEA0432019C43EA0603A4F10C0402949F
:1004E000009CCDE900B400F0E1F803B0BDE8F08F66
:1004F00000200146F9E7C10F80EAE0700844CA070E
:100500009623002100F095B896230022114600F0B2
:1005100090B820F00040C10DC0F3160040F4000078
:100520007F2901DA00207047962903DCC1F196018A
:10053000C8407047963988407047C1F30A5210B5D9
:10054000C1F3130140F2FF3341F480119A4201DA02
:10055000002010BD40F233439A42A2F2334203DC42
:100560005242FFF753FE10BD904010BD00F0004214
:1005700030F000400AD0C10D01F56071C0F31600E3
:1005800042EA0151C208400711437047002001466A
:10059000704701F0004330B421F0004150EA0102FD
:1005A00006D00A0DA2F56072C1F31301002A02DC25
:1005B00030BC00207047440F44EAC104C100E01879
:1005C00030BC00EBC25000F02BB80000002801DB6B
:1005D000C0F10040002901DBC1F1004181427047B8
:1005E000002801DBC0F10040002901DBC1F100411E
:1005F0008842704730B50B46014600202022012476
:1006000009E021FA02F59D4205D303FA02F5491BE0
:1006100004FA02F52844151EA2F10102F1DC30BDF6
:100620000029A8BF7047401C490008BF20F0010006
:10063000704710B4B0FA80FC00FA0CF050EA0104E4
:1006400004BF10BC704749B1CCF1200421FA04F476
:1006500011FA0CF118BF012121430843A3EB0C014F
:10066000CB1D4FEA00614FEA102042BF002010BCB2
:10067000704700EBC35010440029A4BF10BC704762
:10068000401C490008BF20F0010010BC704710B5A5
:10069000141E73F1000408DA401C41F100019218A5
:1006A0005B411A4301D120F0010010BD2DE9F04D4E
:1006B00092469B4611B1B1FA81F202E0B0FA80F2A3
:1006C0002032904600F052F804460F4640EA0A00F5
:1006D00041EA0B0153465A46084313D0114653EAE8
:1006E000010019D0C8F140025046FFF78FFD0546C2
:1006F0000E4650465946424600F038F8084305D0A9
:10070000012004E020463946BDE8F08D0020054375
:1007100046EAE0762C4337430A986305E40AA0EBE7
:1007200008000022FD0A44EA47540A3002D500209E
:100730000146E9E7010510196941DDE9084500199D
:100740006941BDE8F04DA2E7064C074D06E0E068C0
:1007500040F0010394E8070098471034AC42F6D308
:10076000FFF7EAFC8C800008AC800008202A04DB3C
:10077000203A00FA02F1002070479140C2F12003B4
:1007800020FA03F319439040704770B58C1810F8A5
:10079000015B15F0070301D110F8013B2A1106D1C6
:1007A00010F8012B03E010F8016B01F8016B5B1EE0
:1007B000F9D12B0705D40023521E0DD401F8013BBB
:1007C000FAE710F8013BCB1A921C03E013F8015B27
:1007D00001F8015B521EF9D5A142D8D3002070BDAB
:1007E00010B5024800F05FFC10BD00004C0F002067
:1007F00070B5044600252068806800F0010018B339
:100800002068806820F001002168886001F040FDC8
:10081000054613E001F03CFD401B02280ED920687C
:10082000806800F0010048B1A06A40F01000A062AA
:10083000E06A40F00100E062012070BD206880683D
:1008400000F001000028E5D10020F6E738B50446A5
:100850000025002000902068806800F0010078BB2F
:100860002068806840F001002168886019480068AD
:100870001949B0FBF1F0009002E00098401E009092
:1008800000980028F9D101F003FD054619E001F0B8
:10089000FFFC401B022814D92068806800F001008A
:1008A00078B9A06A40F01000A062E06A40F0010050
:1008B000E06200BF002084F8240000BF012038BDA2
:1008C00005E02068806800F001000028DFD00020EB
:1008D000F5E70000A405002040420F0010B51848BD
:1008E00006F084FC17490880174806F07FFC17497A
:1008F0000880144800884FF6FF71884202D01148E2
:10090000008801E012480088114908800F480088DB
:100910004FF6FF71884202D00C48008801E00D4874
:1009200000880C4908800A480088C0F30E00084976
:10093000088008480088C0F30E000649088010BDF2
:10094000001807086C000020002007086E00002037
:100950007E00002080000020F0B597B006460D46CE
:1009600001A803F0C5F8002412E004F500708542E8
:1009700002D94FF4007700E02F1B31193A46114895
:10098000FFF754FC3A460F4901A803F0B1FC3C4480
:10099000AC42EAD301A90C4803F07CF8002407E03C
:1009A0000948005D0949615C884200D002E0641C8E
:1009B000102CF5D300BF102C02D3012017B0F0BDCE
:1009C0000020FBE7002000201E2800200050070820
:1009D000F0B50446187822F810400025002004E005
:1009E00032F810603544461CF0B20A28F8DB0A20C1
:1009F000B5FBF0F008801878401C0A2690FBF6F74B
:100A000006FB17001870F0BD00BFFEE72DE9FC479C
:100A100007460D463846FFF777FD81462946FFF722
:100A200088FC04464FF08B41FFF7B5FC0646314683
:100A30002846FFF778FC814649463046FFF7ABFC75
:100A400004461549FFF775FC8046002419E0134A57
:100A5000601C52F820104046FFF7C2FD10D80F4826
:100A600050F824104046FFF7B1FD09D20A20234672
:100A70000A4A0B49CDE90040404605F03FFE04E03C
:100A8000641C40F247208442E1D300BF054800883F
:100A9000FFF73AFDBDE8FC8700002041CC020020B2
:100AA000840000201805002010B5024800F0F2FE76
:100AB00010BD00004848002010B5024800F0EAFED2
:100AC00010BD00000448002010B5024800F0E2FE0E
:100AD00010BD0000C047002030B590F84050012400
:100AE000AC40C56B6C60046863604468102C04D132
:100AF0000468A2600468E16003E00468A16004681F
:100B0000E26030BD704770B503460024002010E05D
:100B10000E5C451C4D5D46EA0526851C4D5D46EA8A
:100B20000546C51C4D5D46EA056543F82450641C26
:100B3000001D9042ECD370BD70B5034614460022F0
:100B4000002015E011F822501D5431F82250C5F351
:100B50000726451C5E5551F82250C5F30746851CF3
:100B60005E5551F822502D0EC61C9D55521C001D7D
:100B7000A042E7D370BD72B600BFFEE70021074A6E
:100B8000D1610749096941F00401054A1161114623
:100B9000096941F04001116170470000D848002008
:100BA000002002400021074AD1610749096941F04C
:100BB0000201054A116111464861096941F040018D
:100BC00011617047D8480020002002400022054BE8
:100BD000DA61054A126942F00102034B1A61018091
:100BE00070470000D84800200020024000201E4925
:100BF000C96801F0100139B11C49C96941F002010D
:100C00001A4AD16140F010001749C96801F0040187
:100C100039B11649C96941F00101144AD16140F066
:100C200004001149C96901F0010169B10F49C9699D
:100C300041F004010D4AD16100BF0B49C96921F09F
:100C40000101094AD16100BF00BF40F20111884291
:100C500006D10549C96921F00101034AD16101E0CA
:100C60000149C86000BF704700200240D8480020FA
:100C700070B5044601F00CFB054609E0601C38B174
:100C800024B101F005FB401BA04201D9032070BD37
:100C90001248C06800F001000028EFD10F48C0687A
:100CA00000F0200020B100BF20200C49C86000BF28
:100CB0000A48C06800F0100048B90848C06900F050
:100CC000010020B90548C06800F0040018B1FFF722
:100CD0008DFF0120DBE70020D9E700000020024063
:100CE000F0B503461C4600250026084607E010F82C
:100CF000015B10F8016B45EA062724F8027B171EFA
:100D0000A2F1010C1FFA8CF2F1D1F0BD2DE9F047F0
:100D100086B080460E4691464FF0000A0027002517
:100D2000C6F30A0AA6EB0A07002005900190039774
:100D300001200490820239461548FFF7D1FF00BF19
:100D400007E038F8150005EB5A01114A22F81100A6
:100D50006D1C4D45F5D301F0CBF805A901A801F0B4
:100D60000DF800240BE00A4830F814C007EB4401EA
:100D700062460023012001F063F8601C84B2B4F5E0
:100D8000806FF0DB01F052F806B0BDE8F08700009C
:100D9000001000202DE9F04781463A4800F0BEFBE4
:100DA0006421384800F0FAFA364800F078F986B243
:100DB00035493046FFF72AFE8046FFF7AAFB87B287
:100DC000324B334A33493846FFF702FE2D4800F0D4
:100DD000A5FB64212B4800F0E1FA2A4800F05FF9F6
:100DE00085B22D480580B5B12C48008800F400403C
:100DF00010B12B48008802E029480088404228446E
:100E000085B240F68B6027490880084600888542F5
:100E100001DB08460588244B244A25492846FFF76C
:100E2000D7FD184800F07AFB6421164800F0B6FAA6
:100E3000144800F034F984B21E480480B4B11E484E
:100E4000008800F4004010B11C48008802E01B48F4
:100E500000884042204484B240F68B6018490880E4
:100E600008460088844201DB08460488154B164A70
:100E700016492046FFF7ACFD024800F0E7FBBDE84D
:100E8000F08700004C0F00203333534076000020E1
:100E90007C0F0020700000207A0000206C000020F1
:100EA0007E0000201405002077000020900F002015
:100EB000720000207C0000206E00002080000020D6
:100EC0001605002078000020A40F002074000020E8
:100ED0002DE9F041002500241EE0002600270CE04B
:100EE000104A02EBC40291880E4A52F8340004F012
:100EF00099FA304486B2781CC7B20A2FF0DB052E6F
:100F000004DB0120A0402843C5B203E00020A0403C
:100F10002843C5B2601CC4B2082CDEDB2846BDE8FD
:100F2000F0810000747F000802490968C1F3C30022
:100F3000704700000C0C01407047000038B50246B5
:100F400000230020009000BF92F82400012801D166
:100F5000022038BD012082F8240000BF486807281D
:100F600012D21068406B0C79641E04EB84051F24B8
:100F7000AC40A0430D796D1E05EB85050C68AC40B7
:100F800020431468606327E048680D2812D2106877
:100F9000006B0C79E41F04EB84051F24AC40A043D4
:100FA0000D79ED1F05EB85050C68AC4020431468F6
:100FB000206311E01068C06A0C790D3C04EB8405D5
:100FC0001F24AC40A0430D790D3D05EB85050C6851
:100FD000AC4020431468E06208680A2812D3106805
:100FE000C0680C780A3C04EB44050724AC40A043DD
:100FF0000D780A3D05EB45058C68AC40204314682C
:10100000E0600FE0106800690C7804EB44050724E9
:10101000AC40A0430D7805EB45058C68AC402043FF
:10102000146820610868102802D00868112827D1A8
:10103000174C1068A0421ED11068806800F40000B0
:10104000F0B91068806840F400001468A060086877
:10105000102815D10F4800680F4CB0FBF4F000EBDE
:1010600080004000009002E00098401E0090009830
:101070000028F9D104E0906A40F02000906201233A
:1010800000BF002082F8240000BF184661E700007E
:1010900000240140A405002040420F007047014693
:1010A0000868C06C704770B5044620680568206801
:1010B000466806F0200020282DD105F00200022805
:1010C00029D1A06A00F0100018B9A06A40F400709D
:1010D000A0622068806800F46020B0F5602F13D112
:1010E000207B88B92068406820F020002168486093
:1010F000A06A20F48070A062A06A00F4805018B941
:10110000A06A40F00100A0622046FFF7C7FF6FF021
:1011100012002168086006F08000802839D105F0AF
:101120000400042835D1A06A00F0100018B9A06AA4
:1011300040F40050A0622068806800F4E040B0F500
:10114000E04F0DD02068406800F48060D0B920687E
:10115000806800F46020B0F5602F13D1207B88B93F
:101160002068406820F0800021684860A06A20F470
:101170008050A062A06A00F4807018B9A06A40F0A4
:101180000100A0622046FFF7D7FE6FF00C00216837
:10119000086006F0400040280DD105F0010050B174
:1011A000A06A40F48030A062204600F0B5F86FF0ED
:1011B00001002168086070BD2DE9F0410446002758
:1011C00000250026A84614B90120BDE8F081A068DA
:1011D00010B1207D00B100BFA06A30B90020E062EC
:1011E00084F82400204600F099F82046FFF700FB21
:1011F0000746A06A00F01000002873D1002F7ED1AE
:10120000A06A20F4885040F00200A0623F4AD4E96E
:101210000001904208D1E069B0F5402F02D14FF4AF
:10122000002002E0E06900E0E0690143207B41EA40
:1012300040000643A068B0F5807F02D0A068012876
:1012400002D14FF4807000E000200543207D01288A
:1012500011D1207B38B9A069401E4FF4006141EAEA
:101260004030054307E0A06A40F02000A062E06A39
:1012700040F00100E0622068406820F469402843A3
:10128000216848602068806821490840304321680F
:101290008860A068B0F5807F02D0A068012802D1E4
:1012A0004FF4807000E00020B0F5807F03D1208AE9
:1012B000401E4FEA00582068C06A20F4700040EADF
:1012C00008002168C8622068806812490840B0425E
:1012D00009D10020E062A06A20F0020040F0010085
:1012E000A06211E00BE0A06A20F0020040F01000C4
:1012F000A062E06A40F00100E062012704E0A06A19
:1013000040F01000A062012738465EE7003C014033
:10131000FDF7E1FFFE0E1FFF7047000010B586B01D
:10132000044600200290039004900590184920681C
:1013300088422AD100BF1748806940F400701549DF
:1013400088610846806900F40070019000BF00BF0A
:1013500000BF0846806940F0100088610846806937
:1013600000F01000019000BF00BF07200290032092
:10137000039002A9084800F0D3FD002205211220A5
:1013800001F046F8122001F033F806B010BD00005D
:10139000002401400010024000100140F8B504464E
:1013A0000D46002600200090002700F071FF064641
:1013B0002068806800F4807050B1A06A40F020007E
:1013C000A06200BF002084F8240000BF0120F8BD07
:1013D0002068406800F4807020BB2068C06A00F478
:1013E0007000F8B917E0681CA8B125B100F050FFF3
:1013F000801BA8420FD92068006800F0020050B995
:10140000A06A40F00400A06200BF002084F824001D
:1014100000BF0320DBE72068006800F0020000281E
:10142000E1D053E0022001F067F838490968B1FBC8
:10143000F0F021680969364A114091B92168C968FC
:101440009211114069B921680969324A114031B9D4
:101450002168C9689211114009B9142117E02921A6
:1014600015E0216809692B4A114021B92168C96832
:101470009211114041B121680969274A114029B9E7
:101480002168C968114009B9542100E0FC2100FB22
:1014900001F718E0681C98B125B100F0F9FE801B37
:1014A000A8420DD90098B8420AD2A06A40F00400C0
:1014B000A06200BF002084F8240000BF032086E75C
:1014C0000098401C00900098B842E3D36FF01200DF
:1014D00021680860A06A40F40070A06220688068FB
:1014E00000F46020B0F5602F0DD1207B58B9A06AC0
:1014F00020F48070A062A06A00F4805018B9A06A3D
:1015000040F00100A062002061E70000A405002077
:1015100024499224922449124992240070B5044629
:10152000002500BF94F82400012801D1022070BDDD
:10153000012084F8240000BF2046FFF787F9054604
:10154000002D77D1A06A40F20121884340F48070D9
:10155000A0623C492068884208D13B48006800F4FA
:10156000702008B9012002E0002000E0012078B1DD
:10157000A06A20F48010A0622068406800F48060B7
:1015800000B3A06A20F4005040F48050A06219E03B
:10159000A06A40F48010A0622B49091F206888428D
:1015A00003D028492068884204D12748006800F405
:1015B000806000E0002028B1A06A20F4005040F4D0
:1015C0008050A062A06A00F4805020B1E06A20F050
:1015D0000600E06201E00020E06200BF002084F825
:1015E000240000BFC01E216808602068806800F4E5
:1015F0006020B0F5602F16D112492068884208D1CA
:101600001148006800F4702008B9012002E00020B1
:1016100000E0012038B12068806840F4A000216813
:1016200088600CE006E02068806840F48010216843
:10163000886004E000BF002084F8240000BF284632
:1016400075E70000002801400424014070B50446FD
:10165000002500BF94F82400012801D1022070BDAC
:10166000012084F8240000BF2046FFF7C1F805469A
:101670002DB9A06A20F4885040F00100A06200BF9C
:10168000002084F8240000BF2846E8E70146002235
:1016900091F82100022808D00420886300BF0020B0
:1016A00081F8200000BF012070470868006820F022
:1016B0000E000B6818600868006820F001000B68D5
:1016C000186091F8403001209840CB6B58600120A1
:1016D00081F8210000BF002081F8200000BF1046E3
:1016E000E2E7000070B50446002594F821000228C6
:1016F00003D00420A0630125C1E02068006820F029
:101700000E00216808602068006820F00100216850
:1017100008605C492068884252D95A497839206863
:10172000884201D1012047E0564964392068884247
:1017300001D1102040E0534950392068884201D13E
:10174000801539E04F493C392068884201D1801426
:1017500032E04C4928392068884202D14FF4803069
:101760002AE0484914392068884202D14FF4801099
:1017700022E044492068884201D140041CE04249EB
:101780002068884201D1012016E03F4914312068C9
:10179000884201D110200FE03B492831206888425F
:1017A00001D1801508E038493C312068884201D1D8
:1017B000801401E04FF480303349091F086051E084
:1017C000304978392068884201D1012047E02D490D
:1017D00064392068884201D1102040E029495039FD
:1017E0002068884201D1801539E026493C392068BB
:1017F000884201D1801432E0224928392068884289
:1018000002D14FF480302AE01E4914392068884202
:1018100002D14FF4801022E01A492068884201D199
:1018200040041CE018492068884201D1012016E0DC
:10183000154914312068884201D110200FE0124967
:1018400028312068884201D1801508E00E493C31DA
:101850002068884201D1801401E04FF480300949AA
:1018600080394860012084F8210000BF002084F8FE
:10187000200000BF606B10B12046616B884728468E
:1018800070BD000080000240080402400146886BE1
:101890007047000070B50446E06B05682068066874
:1018A00094F84010042088402840002875D006F0A5
:1018B00004000028FAD02068006800F0200028B951
:1018C0002068006820F0040021680860D54920687D
:1018D000884254D9D34978392068884201D10420FC
:1018E00049E0D04964392068884201D1402042E073
:1018F000CC4950392068884201D100153BE0C949E4
:101900003C392068884202D14FF4804033E0C54919
:1019100028392068884202D14FF480202BE0C14949
:1019200014392068884202D14FF4800023E0BD4979
:101930002068884201D1C0041DE0BB49206888426C
:1019400001D1042017E0B84914312068884201D140
:10195000402010E0B44928312068884201D10015A8
:1019600009E0B1493C312068884202D14FF48040FF
:1019700001E04FF48020AC49091F086054E0A949F8
:1019800078392068884201D104204AE0A5496439A9
:101990002068884202D1402043E04CE0A149503900
:1019A0002068884201D100153BE09E493C392068FF
:1019B000884202D14FF4804033E09A4928392068A8
:1019C000884202D14FF480202BE0964914392068D8
:1019D000884202D14FF4800023E092492068884277
:1019E00001D1C0041DE090492068884201D1042043
:1019F00017E08D4914312068884201D1402010E061
:101A0000894928312068884201D1001509E08649BA
:101A10003C312068884202D14FF4804001E04FF40D
:101A20008020804980394860E06A002802D0204642
:101A3000E16A8847F4E094F840100220884028408A
:101A4000002871D006F002000028FAD02068006853
:101A500000F0200040B92068006820F00A002168EA
:101A60000860012084F821006E492068884254D91A
:101A70006C4978392068884201D1022049E06949DF
:101A800064392068884201D1202042E065495039FC
:101A90002068884201D140153BE062493C3920680A
:101AA000884202D14FF4005033E05E492839206863
:101AB000884202D14FF400302BE05A491439206893
:101AC000884202D14FF4001023E056492068884232
:101AD00001D180041DE054492068884201D10220D0
:101AE00017E0514914312068884201D1202010E0CC
:101AF0004D4928312068884201D1401509E04A4902
:101B00003C312068884202D14FF4005001E04FF48C
:101B100000304549091F086054E04249783920687F
:101B2000884202D102204AE057E03E4964392068E9
:101B3000884201D1202042E03A4950392068884249
:101B400001D140153BE037493C392068884202D139
:101B50004FF4005033E0334928392068884202D1DD
:101B60004FF400302BE02F4914392068884202D10D
:101B70004FF4001023E02B492068884201D18004F3
:101B80001DE029492068884201D1022017E026493A
:101B900014312068884201D1202010E022492831E8
:101BA0002068884201D1401509E01F493C31206876
:101BB000884202D14FF4005001E04FF4003019493F
:101BC0008039486000BF002084F8200000BFA06A70
:101BD00030B32046A16A884722E094F840100820DC
:101BE00088402840E0B106F00800C8B120680068CD
:101BF00020F00E002168086094F840100120884011
:101C0000E16B48600120A06384F8210000BF002040
:101C100084F8200000BF206B10B12046216B88475C
:101C200070BD00008000024008040240014600220E
:101C300009B9012070471E4B086898420BD21D4B12
:101C40000868C01A1423B0FBF3F080000864194838
:101C50000838C8630AE0164B0868C01A1423B0FBA2
:101C6000F3F08000086412480838C863022081F845
:101C700021000868026843F6F0708243D1E901034D
:101C80001843CB6818430B6918434B6918438B6999
:101C90001843CB6918430243086802600020886338
:101CA000012081F82100002081F8200000BFC1E759
:101CB00008040240080002402DE9F04104460D46A8
:101CC00016461F464FF0000800BF94F82000012878
:101CD00002D10220BDE8F081012084F8200000BF7D
:101CE00094F8210001282CD1022084F82100002042
:101CF000A0632068006820F00100216808603B466E
:101D0000324629462046FEF7E7FEE06A30B12068F9
:101D1000006840F00E00216808600BE02068006851
:101D200020F00400216808602068006840F00A0084
:101D3000216808602068006840F0010021680860A0
:101D400006E000BF002084F8200000BF4FF002082A
:101D50004046BFE770B5044600F09AFA06462546AD
:101D6000681C10B104480078054400BF00F090FAE8
:101D7000801BA842FAD370BDA00500202DE9F041D8
:101D800004460E460127002500BF2648007E012894
:101D900002D10220BDE8F08101202249087600BF6F
:101DA0002068022813D14CF25030FEF761FF90BB3F
:101DB0000120FEF7E3FE4CF25030FEF759FF0746D4
:101DC0001948006920F004001749086123E04CF22B
:101DD0005030FEF74DFFF0B94FF0FF303060A5688E
:101DE00012E02846FEF7DEFE4CF25030FEF740FFD0
:101DF00007460D48006920F002000B4908610FB149
:101E0000356007E005F50065D4E9021001EBC0205C
:101E1000A842E6D800BF00BF00200249087600BFF4
:101E20003846B7E7D8480020002002400348006940
:101E300040F0800001490861002070470020024006
:101E40002DE9FE4F05468B4617469846012600248D
:101E50000020029000BF2448007E012802D1022009
:101E6000BDE8FE8F01202049087600BF4CF25030BB
:101E7000FEF7FEFE064686BB012D02D10120029030
:101E800006E0022D02D10220029001E0042002901F
:101E900000241EE02201B946C24648465146FEF7DC
:101EA000B5F980B20190022000FB04B000900199C6
:101EB000FEF78CFE4CF25030FEF7DAFE06460B4879
:101EC000006920F001000949086106B104E0601CC6
:101ED000C4B202988442DDDB00BF00BF002002498B
:101EE000087600BF3046BBE7D848002000200240FB
:101EF00000200849096901F0800151B10649054AED
:101F00005160064951601146096901F0800101B133
:101F1000012070470020024023016745AB89EFCDC7
:101F20002DE9F847024600239C467BE14FF001086B
:101F300008FA03F4D1F8008008EA0400A0427DD139
:101F4000DFF8F4A2D1F80480A8EB0A09D0453AD012
:101F500014DCB8F1030F50D009DCB8F1000F31D018
:101F6000B8F1010F1CD0B8F1020F49D120E0B8F14F
:101F7000110F18D0B8F1120F42D11EE0B9F5881F29
:101F800025D006DCB9F5803F20D0B9F5801F37D1C8
:101F90001AE0B9F5001F18D0B9F5041F30D117E0C9
:101FA000D1F80CC02DE0D1F80C8008F1040C28E029
:101FB000D1F80C8008F1080C23E0D1F80C8008F16E
:101FC0000C0C1EE000BF00BF00BF00BF00BF00BF81
:101FD000D1F80880B8F1000F02D14FF0040C0BE0EB
:101FE000D1F80880B8F1010F03D14FF0080C14614B
:101FF00002E04FF0080C546103E04FF0000C00E0E9
:1020000000BF00BFFF2801D8904601E002F104089C
:102010004646FF2802D84FEA830803E0A3F10808E8
:102020004FEA88084746D6F800804FF00F0909FAB2
:1020300007F928EA09080CFA07F900E07AE048EA0B
:102040000908C6F80080D1F8048008F08058B8F17B
:10205000805F6FD100BFDFF8E481D8F8188048F0C6
:102060000108DFF8D891C9F81880C846D8F8188058
:1020700008F00108CDF8008000BF00BF4FEAB93872
:102080004FEA930958F829504FEA83784FEA1879B4
:102090004FF00F0808FA09F825EA0805DFF8A081D3
:1020A000424502D14FF0000824E0DFF89881424514
:1020B00002D14FF001081DE0DFF88C81424502D1CA
:1020C0004FF0020816E0DFF88481424502D14FF05C
:1020D00003080FE0DFF87881424502D14FF0040891
:1020E00008E0DFF87081424502D14FF0050801E0B9
:1020F0004FF006084FEA83794FEA197908FA09F890
:1021000048EA0505DFF850814FEA930948F829505D
:10211000D1F8048008F48018B8F5801F0BD1DFF8DF
:102120003C81D8F8008048EA0008DFF83091C9F80F
:1021300000800AE075E0DFF82481D8F8008028EA02
:102140000008DFF81891C9F80080D1F8048008F47D
:102150000018B8F5001F0ED1DFF8008108F104085F
:10216000D8F8008048EA0008DFF8F09009F1040987
:10217000C9F800800DE0DFF8E48008F10408D8F821
:10218000008028EA0008DFF8D49009F10409C9F8B2
:102190000080D1F8048008F40038B8F5003F0ED173
:1021A000DFF8B880A8F10408D8F8008048EA0008F1
:1021B000DFF8A890A9F10409C9F800800DE0DFF864
:1021C0009C80A8F10408D8F8008028EA0008DFF80D
:1021D0008C90A9F10409C9F80080D1F8048008F4B2
:1021E0008038B8F5803F0ED1DFF87080A8F108087C
:1021F000D8F8008048EA0008DFF86090A9F10809E3
:10220000C9F800800DE0DFF85480A8F10808D8F87C
:10221000008028EA0008DFF84490A9F10809C9F80D
:1022200000805B1CD1F8008028FA03F8B8F1000F99
:102230007FF47CAEBDE8F88700001110001002406A
:1022400000080140000C0140001001400014014052
:1022500000180140001C0140080001400804014032
:10226000024693680B400BB1012000E0002070474C
:1022700010B5C26821EA020302EA010443EA0443FA
:10228000036110BD0AB1016101E00B0403617047F5
:102290000148006870470000980500200348006866
:1022A00003490978084401490860704798050020EF
:1022B000A005002010B50848006840F0100006494D
:1022C0000860032000F0E2F80F2000F007F800F0AB
:1022D0005FF8002010BD0000002002402DE9F04111
:1022E00088B004460027B846002600BF2348C069CE
:1022F00040F002002149C8610846C06900F00200B0
:10230000019000BF00BF02A903A800F0DFFA069FFA
:102310001FB900F003FB054602E000F0FFFA45009C
:102320001748B5FBF0F0A0F10108164816490860FF
:1023300040F2E7311448C160C0F804800021016117
:102340008160816100F0C4FD064696B90E4800F038
:1023500013FE06466EB91D2000F04AF8102C07D275
:10236000002221461D2000F053F80848046000E0D8
:102370000126304608B0BDE8F081000000100240A0
:1023800040420F00000400408C4800209C050020C3
:1023900008B500BF1448806940F001001249886107
:1023A0000846806900F00100009000BF00BF00BF38
:1023B0000846C06940F08050C8610846C06900F016
:1023C0008050009000BF00BF00220F21901E00F03F
:1023D0001FF800BF0549486820F0E06040F0007039
:1023E000486000BF08BD000000100240000001402E
:1023F00001460846002809DB00F01F0301229A402D
:1024000043099B0003F1E023C3F8002100BF70479C
:102410002DE9F05F80460D461646002703F094FE36
:10242000074639462A46334601F00700C0F1070A3D
:10243000BAF1040F02D94FF0040A01E0C0F1070A13
:10244000D14600F1040ABAF1070F02D24FF0000A98
:1024500001E0A0F1030AD4464FF0010A0AFA09FA92
:10246000AAF1010A0AEA020A0AFA0CFA4FF0010B71
:102470000BFA0CFBABF1010B0BEA030B4AEA0B0462
:102480002146404603F068FEBDE8F09F00BF00F023
:102490000702064B19684FF6FF031940044B0B4324
:1024A00043EA0221014B196000BF70470CED00E0C8
:1024B0000000FA0500BF00BF00BF00BF00BFBFF3B0
:1024C0004F8F00BF00BF00BF0948006800F4E06004
:1024D00008490843001D0649086000BF00BF00BF4F
:1024E000BFF34F8F00BF00BF00BF00BF00BFFDE7BD
:1024F0000CED00E00000FA052DE9F04706464FF02C
:102500000008002500270024A146042E37D004DC53
:10251000012E3CD0022E6CD160E0082E33D0102E5C
:1025200067D136484468006800F0807008B33448CA
:10253000C4F38341475C04F4803078B12F4840688D
:10254000C0F340402F4911F8008004F4803040B1BE
:102550002D48B0FBF8F000FB07F502E02B4807FB25
:1025600000F52648406800F48000B0F5800F01D1E6
:10257000A94603E068000321B0FBF1F93AE000F05E
:10258000EDF9814636E000F0E9F9814632E01B487A
:10259000046A04F44070B0F5807F05D104F00200B5
:1025A00010B14FF4004918E004F44070B0F5007F1A
:1025B00007D11248406A00F0020010B149F64049C4
:1025C0000BE004F44070B0F5407F06D10B48006882
:1025D00000F4003008B14FF224490BE000F0AEF9EE
:1025E00006494968C1F38131491C4900B0FBF1F942
:1025F00000E000BF00BF4846BDE8F0870010024081
:10260000368000084680000800127A0000093D006C
:10261000F8B5044600260025207800F001000028C7
:102620006BD000274348C06900F0805070B900BFEC
:102630004048C06940F080503E49C8610846C069C2
:1026400000F08050009000BF00BF01273A480068AA
:1026500000F48070B0B93848006840F480703649A2
:102660000860FFF715FE064606E0FFF711FE801B27
:10267000642801D90320F8BD2F48006800F4807059
:102680000028F2D02B48006A00F440752DB3A088D2
:1026900000F44070A84220D02648006A20F440751B
:1026A000012026490860002008602248056205F0E4
:1026B000010090B1FFF7ECFD064608E0FFF7E8FDEA
:1026C000801B41F28831884201D90320D3E71948A1
:1026D000006A00F002000028F0D01648006A20F4DA
:1026E00040706168084313490862012F04D108460D
:1026F000C06920F08050C86100BF207800F002005F
:10270000022807D10B48406820F44040A1680843E4
:1027100008494860207800F01000102807D10548CB
:10272000406820F480006169084302494860002045
:10273000A1E7000000100240007000404004424247
:1027400070B504460D460CB9012070BD5A480068AA
:1027500000F00700A8420ED25748006820F007009A
:102760002843554908600846006800F00700A84261
:1027700001D00120E9E7207800F0020002281DD1F5
:10278000207800F00400042805D14C48406840F44B
:10279000E0604A494860207800F00800082805D128
:1027A0004648406840F460504449486043484068A7
:1027B00020F0F000A168084340494860207800F00C
:1027C000010078B36068012806D13C48006800F435
:1027D000003090B90120B8E76068022806D1374878
:1027E000006800F0007040B90120AEE7334800688F
:1027F00000F0020008B90120A7E73048406820F047
:102800000300616808432D494860FFF741FD064613
:1028100009E0FFF73DFD801B41F28831884202D973
:10282000032092E707E02548406800F00C0061684B
:10283000B0EB810FEDD12048006800F00700A842FE
:102840000ED91D48006820F0070028431A49086087
:102850000846006800F00700A84201D0012074E794
:10286000207800F00400042807D11448406820F4C0
:10287000E060E168084311494860207800F00800F2
:10288000082808D10D48406820F46050216940EACA
:10289000C1000A49486000F061F808494968C1F37D
:1028A0000311074A515CC8400649086006480068A1
:1028B000FFF714FD002048E700200240001002400E
:1028C00048800008A40500209C0500200F2202601B
:1028D0000D4A526802F0030242600B4A526802F04D
:1028E000F0028260084A526802F4E062C260064A5E
:1028F000526802F46052D2080261044A126802F07F
:1029000007020A60704700000010024000200240E9
:102910000148006870470000A405002000B5FFF7DB
:10292000F7FF04494968C1F30221034A515CC840DA
:1029300000BD0000001002405880000800B5FFF7FD
:10294000E7FF04494968C1F3C221034A515CC8400A
:1029500000BD0000001002405880000870B5002142
:102960000022002400230020134D696801F00C05AB
:10297000F5B1042D02D0082D19D101E00F4819E05E
:102980000F4DC1F38346AB5D01F4803555B10A4D5F
:102990006D68C5F340450B4E725D084D5D43B5FB58
:1029A000F2F402E0084D03FB05F4204602E000BF0C
:1029B000024800BF00BF70BD0010024000127A0044
:1029C000248000083480000800093D00F8B5044662
:1029D0000CB90120F8BD207800F00100002878D063
:1029E000F848406800F00C0004280CD0F548406816
:1029F00000F00C00082811D1F248406800F4803043
:102A0000B0F5803F0AD1EF48006800F4003000289C
:102A10005FD0606800285CD10120DBE700BF606800
:102A2000B0F5803F06D1E748006840F48030E549C2
:102A3000086028E0606858B9E248006820F48030F7
:102A4000E04908600846006820F4802008601AE029
:102A50006068B0F5A02F0BD1DA48006840F4802000
:102A6000D84908600846006840F4803008600AE0F1
:102A7000D448006820F48030D249086008460068D5
:102A800020F48020086000BF606888B1FFF700FC78
:102A9000054606E0FFF7FCFB401B642801D9032034
:102AA00098E7C848006800F400300028F2D010E031
:102AB000FFF7EEFB054606E0FFF7EAFB401B642844
:102AC00001D9032086E7BF48006800F400300028E1
:102AD000F2D1207800F00200022857D1B9484068AE
:102AE00000F00C0050B1B748406800F00C00082816
:102AF00018D1B448406800F4803098B9B1480068F3
:102B000000F0020020B12069012801D0012061E716
:102B1000AC48006820F0F800616940EAC100A949AA
:102B2000086033E02069E8B10120A7490860FFF799
:102B3000AFFB054606E0FFF7ABFB401B022801D9BF
:102B4000032047E79F48006800F002000028F2D009
:102B50009C48006820F0F800616940EAC10099498A
:102B6000086013E0002098490860FFF791FB0546D4
:102B700006E0FFF78DFB401B022801D9032029E75F
:102B80009048006800F002000028F2D1207800F0A0
:102B9000080008282DD1A069B8B101208B49086030
:102BA000FFF776FB054606E0FFF772FB401B0228A5
:102BB00001D903200EE78348406A00F00200002894
:102BC000F2D0012002F01AFC13E000207F490860D7
:102BD000FFF75EFB054606E0FFF75AFB401B0228A5
:102BE00001D90320F6E67748406A00F00200002889
:102BF000F2D1207800F00400042873D10027714836
:102C0000C06900F0805070B900BF6E48C06940F0E4
:102C100080506C49C8610846C06900F0805000903F
:102C200000BF00BF01276A48006800F48070B0B997
:102C30006748006840F4807065490860FFF728FB2A
:102C4000054606E0FFF724FB401B642801D903205A
:102C5000C0E65F48006800F480700028F2D000BF32
:102C6000E068012806D15748006A40F00100554944
:102C7000086227E0E06858B95248006A20F0010075
:102C8000504908620846006A20F00400086219E012
:102C9000E06805280BD14B48006A40F00400494920
:102CA00008620846006A40F0010008620AE04548F0
:102CB000006A20F00100434908620846006A20F0DB
:102CC0000400086200BFE068A0B1FFF7E1FA054622
:102CD00009E0FFF7DDFA401B41F28831884202D952
:102CE000032077E622E03748006A00F0020000285F
:102CF000EFD012E0FFF7CCFA054608E0FFF7C8FA7C
:102D0000401B41F28831884201D9032062E62D48F8
:102D1000006A00F002000028F0D1012F05D12948F7
:102D2000C06920F080502749C86100BFE069C8B37E
:102D30002448406800F00C00082860D0E0690228B0
:102D400048D1002020490866FFF7A2FA054606E0B0
:102D5000FFF79EFA401B022801D903203AE61948E2
:102D6000006800F000700028F2D1206AB0F5803FC2
:102D700007D11448406820F40030A1680843114985
:102D80004860D4E9080108430E49496821F47411E8
:102D900008430C49486001200B490866FFF778FAA0
:102DA000054607E03DE0FFF773FA401B022801D912
:102DB00003200FE60348006800F000700028F2D0FE
:102DC0002FE0000000100240000042428004424216
:102DD00000700040002014490866FFF759FA0546C4
:102DE00006E0FFF755FA401B022801D90320F1E560
:102DF0000E48006800F000700028F2D111E0E06990
:102E0000012800D1E6E50948466806F48031206AC9
:102E1000814204D106F47011606A814201D0012020
:102E2000D8E50020D6E50000000042420010024034
:102E30007047704730B502460B4600BF92F83C0021
:102E4000012801D1022030BD012082F83C0000BFE2
:102E5000022082F83D00106844681068816824F000
:102E600070041868044310684460144D1068A84248
:102E700013D0134D1068A8420FD01068B0F1804FE6
:102E80000BD0104D1068A84207D00F4D1068A84213
:102E900003D00E4D1068A84205D121F0800158687A
:102EA000014310688160012082F83D0000BF0020CE
:102EB00082F83C0000BF00BFC5E70000002C0140C5
:102EC000003401400004004000080040000C0040B5
:102ED00010B504460CB9012010BD94F83D0028B986
:102EE000002084F83C00204600F026F8022084F8F8
:102EF0003D00211D206802F0BBFC012084F8460043
:102F000000BF84F83E0001213F20015540200155BB
:102F10004120015500BF00BF012084F8420043203A
:102F20000155442001554520015500BF012084F87A
:102F30003D000020D0E7000038B504462068B0F11D
:102F4000804F15D100BF0B48C06940F0010009490E
:102F5000C8610846C06900F00100009000BF00BFD2
:102F6000002205211C20FFF753FA1C20FFF740FA2E
:102F700038BD000000100240014691F83D000128D4
:102F800001D001207047022081F83D000868C06828
:102F900040F001000B68D860164B0868984213D0C7
:102FA000154B086898420FD00868B0F1804F0BD0DD
:102FB000124B0868984207D0114B0868984203D01A
:102FC000104B086898420CD10868806800F007022E
:102FD000062A0CD00868006840F001000B681860F1
:102FE00005E00868006840F001000B6818600020E8
:102FF000C8E70000002C01400034014000040040FC
:1030000000080040000C00402DE9F04104460D4648
:10301000002700BF94F83C00012802D10220BDE83F
:10302000F081012084F83C0000BF022084F83D00BC
:103030002068866826F0770626F47F46206886603A
:103040002868502833D00CDC202850D004DC00281D
:103050004BD0102851D149E0302849D040284CD1DC
:1030600039E060282DD0702807D0B0F5805F03D0FC
:10307000B0F5005F41D10DE041E0D5E902136A6887
:10308000206802F043FC2068866846F077062068D6
:10309000866034E0D5E902136A68206802F036FCE5
:1030A0002068806840F480402168886027E0EA68F2
:1030B0006968206802F03EFC5021206802F031FC73
:1030C0001DE0EA686968206802F047FC602120681A
:1030D00002F027FC13E0EA686968206802F02AFC25
:1030E0004021206802F01DFC09E000BF00BF00BFC6
:1030F0002968206802F015FC01E0012700BF00BF2D
:10310000012084F83D0000BF002084F83C0000BF8F
:10311000384684E7704710B5044620680069C0F35C
:103120004000D8B12068C068C0F34000B0B16FF073
:10313000020021680861012020772068806900F082
:10314000030018B12046FFF7E5FF05E0204600F038
:10315000ADF8204600F0ABF8002020772068006929
:10316000C0F38000D8B12068C068C0F38000B0B15F
:103170006FF00400216808610220207720688069D0
:1031800000F4407018B12046FFF7C4FF05E0204668
:1031900000F08CF8204600F08AF8002020772068A4
:1031A0000069C0F3C000D8B12068C068C0F3C00097
:1031B000B0B16FF008002168086104202077206812
:1031C000C06900F0030018B12046FFF7A3FF05E037
:1031D000204600F06BF8204600F069F800202077C8
:1031E00020680069C0F30010D8B12068C068C0F33F
:1031F0000010B0B16FF0100021680861082020773E
:103200002068C06900F4407018B12046FFF782FFC3
:1032100005E0204600F04AF8204600F048F800207B
:1032200020772068006900F0010058B12068C0686C
:1032300000F0010030B16FF0010021680861204604
:1032400000F036F820680069C0F3C01058B120685B
:10325000C068C0F3C01030B16FF080002168086111
:103260002046FFF7E5FD20680069C0F3801058B1E3
:103270002068C068C0F3801030B16FF04000216852
:103280000861204600F020F820680069C0F3401073
:1032900058B12068C068C0F3401030B16FF0200012
:1032A000216808612046FFF7C4FD10BD70477047D4
:1032B00010B5044603492068884201D1FEF7EEFFAD
:1032C00010BD0000000400407047704710B5044670
:1032D00000BF00BF21680C3151E8001F21F490703D
:1032E00021680C3141E80002002AF3D100BF00BF81
:1032F00000BF2168143151E8001F21F0010021684E
:10330000143141E80002002AF3D100BF206B0128EC
:103310000ED100BF00BF21680C3151E8001F21F021
:10332000100021680C3141E80002002AF3D100BFEF
:103330002068406900F0400000B300BF00BF216872
:10334000143151E8001F21F040002168143141E898
:103350000002002AF3D100BFE06B78B10020E16BDE
:103360004863E06BFEF792F940B1E06BFEF78EFA2E
:10337000202803D110206064032010BD0020E085C8
:10338000202084F842000020206300BFF5E770B5DC
:103390000446002520684069C0F3C01594F8410038
:1033A000212817D1B5B100BF00BF2168143151E801
:1033B000001F21F080002168143141E80002002A3A
:1033C000F3D100BFA06B10B1A06BFEF75FF92046F0
:1033D00002F0BBFB20684069C0F3801594F84200FE
:1033E000222817D1B5B100BF00BF2168143151E8C0
:1033F000001F21F040002168143141E80002002A3A
:10340000F3D100BFE06B10B1E06BFEF73FF920464F
:1034100002F055FB002070BD704700002DE9F84F09
:103420000446206805682068C668206847694FF030
:103430000009CA4605F00F09B9F1000F0AD105F0DD
:10344000200038B106F0200020B1204602F090FBA9
:10345000BDE8F88FB9F1000F7BD007F0010018B973
:1034600006F49070002874D005F0010030B106F425
:10347000807018B1606C40F00100606405F00400D9
:1034800030B107F0010018B1606C40F002006064D8
:1034900005F0020030B107F0010018B1606C40F097
:1034A0000400606405F0080048B106F0200010B97F
:1034B00007F0010018B1606C40F008006064606CB7
:1034C000002845D005F0200028B106F0200010B1FA
:1034D000204602F04DFB20684069C0F3801A606C02
:1034E00000F0080010B9BAF1000F2CD0204602F00D
:1034F000E6FA2068406900F0400000B300BF00BF5A
:103500002168143151E8001F21F040002168143176
:1035100041E80002002AF3D100BFE06B50B17748C8
:10352000E16B4863E06BFEF7DDF888B1E06B416B5F
:1035300088470DE02046FFF76FFF09E009E02046CD
:10354000FFF76AFF04E02046FFF766FF0020606493
:103550007EE7206B012877D105F01000002873D09A
:1035600006F010000028FAD000BF0020009020686C
:103570000068009020684068009000BF00BF20688D
:10358000406900F0400000285FD0E06B00684068B0
:103590001FFA80F8B8F1000F55D0A08D404552DDDC
:1035A000A4F82E80E06B8069202843D000BF00BFC4
:1035B00021680C3151E8001F21F4807021680C3122
:1035C00041E80002002AF3D100BF00BF00BF21681C
:1035D000143151E8001F21F001002168143141E845
:1035E0000002002AF3D100BF00BF00BF21681431E0
:1035F00051E8001F21F040002168143141E8000229
:10360000002AF3D100BF202084F84200002020636C
:1036100000BF00BF21680C3151E8001F21F01000ED
:1036200021680C3141E80002002AF3D100BFE06BB1
:10363000FEF72CF802206063A08DE28D801A81B223
:103640002046FFF742FE03E742E0A08DE18D401ADD
:103650001FFA80F8E08DD0B3B8F1000F37D000BF6B
:1036600000BF21680C3151E8001F21F490702168DF
:103670000C3141E80002002AF3D100BF00BF00BFB7
:103680002168143151E8001F21F001002168143134
:1036900041E80002002AF3D100BF202084F8420054
:1036A0000020206300BF00BF21680C3151E8001FDB
:1036B00021F0100021680C3141E80002002AF3D10A
:1036C00000BF0220606341462046FFF7FEFDBFE6D3
:1036D00005F0800030B106F0800018B1204602F0FD
:1036E000A7FBB5E605F0400030B106F0400018B188
:1036F000204602F01AFAABE600BFA9E6835900089B
:1037000010B504460CB9012010BDA06900B100E05D
:1037100000BF94F8410028B9002084F840002046FA
:1037200000F02AF8242084F841002068C06820F4C2
:1037300000502168C860204602F098FA20680069AD
:1037400020F49040216808612068406920F02A0038
:10375000216848612068C06840F400502168C86052
:1037600000206064202084F8410084F8420000209A
:10377000606300BFC8E7000010B586B004460020B3
:1037800002900390049005906249206888426AD1B3
:1037900000BF6148806940F480405F498861084605
:1037A000806900F48040019000BF00BF00BF084660
:1037B000806940F0040088610846806900F00400D8
:1037C000019000BF00BF4815029002200390032023
:1037D000059002A95148FEF7A3FB4FF480600290C8
:1037E00000200390049002A94C48FEF799FB4C4836
:1037F0004C4908600020486000214A4881608021CF
:10380000C1600021016141618161C161FEF70EFA71
:1038100008B1FDF7B0F900BF4248E063446200BF61
:103820003F481438404908601020486000213E4855
:1038300081608021C1600021016141618161C161BC
:10384000FEF7F4F908B1FDF796F900BF3648A0631A
:10385000446200BF002205212520FEF7D9FD252066
:10386000FEF7C6FD54E031492068884250D100BFC0
:103870002948C06940F480202749C8610846C069CA
:1038800000F48020019000BF00BF00BF084680699F
:1038900040F0080088610846806900F00800019047
:1038A00000BF00BF0815029002200390032005907E
:1038B00002A91F48FEF734FB4FF40060029000207D
:1038C0000390049002A91A48FEF72AFB14482838EE
:1038D0001849086000204860002116488160802156
:1038E000C1600021016141618161C161FEF79EF902
:1038F00008B1FDF740F900BF0E48E063446200BF25
:10390000002205212720FEF783FD2720FEF770FD0A
:1039100006B010BD00380140001002400008014010
:1039200058000240C04700200448002000480040E2
:10393000000C01404848002070B504460D4616466C
:1039400094F8420020280BD105B10EB9012070BDBA
:103950000020206332462946204602F005FAF6E7A9
:103960000220F4E76FF020010268116089100268FC
:103970001160704770472DE9F84F04460E46174610
:1039800099464FF0000A94F8410020284AD106B128
:1039900017B90120BDE8F88F00206064212084F869
:1039A0004100FEF775FC8246A784E784A068B0F565
:1039B000805F04D1206910B90025B04602E0354689
:1039C0004FF000081BE05346002280212046CDF82E
:1039D000009002F05DFA08B10320DBE745B9B8F8C2
:1039E0000000C0F308002168486008F1020803E005
:1039F0002878216848606D1CE08C401EE084E08CD3
:103A00000028E0D15346002240212046CDF8009006
:103A100002F03EFA08B10320BCE7202084F8410000
:103A20000020B7E70220B5E710B5034693F8410040
:103A3000202813D101B10AB9012010BD19629A845E
:103A4000DA8400205864212083F841001868C06897
:103A500040F080001C68E0600020EEE70220ECE708
:103A60006FF02001026811608910026811607047D0
:103A700000BFFEE770B50446206805490840B0F174
:103A8000005F04D165682068FCF75EFBA84770BD45
:103A90000000FE2F2DE9FC4106460C46082204F1E9
:103AA00010016846FDF748F8208AC0F3C505382D97
:103AB00002D2C5F1380001E0C5F1780007463A4668
:103AC0000A49204600F014FC08226946204600F00E
:103AD0000FFC102221463046FDF72EF85822002117
:103AE000204600F051FCBDE8FC8100005805002094
:103AF00000224261026105490160054941600349B4
:103B0000C94381600249C943C160704701234567C9
:103B100089ABCDEF2DE9F04391B080468946D8F8C6
:103B20000040D8F80450D8F80860D8F80C7040224B
:103B3000494601A8FCF7E7FF05EA060027EA050168
:103B4000084301990844FE4908440444E00140EA5E
:103B500054642C4404EA050026EA0401084302994F
:103B60000844F84908440744380340EA17572744F3
:103B700007EA040025EA0701084303990844F249CB
:103B800008440644700440EAD6363E4406EA07007C
:103B900024EA0601084304990844EC490844054412
:103BA000A80540EA9525354405EA060027EA0501FF
:103BB000084305990844E64908440444E00140EA02
:103BC00054642C4404EA050026EA040108430699DB
:103BD0000844E04908440744380340EA175727449B
:103BE00007EA040025EA0701084307990844DA496F
:103BF00008440644700440EAD6363E4406EA07000C
:103C000024EA0601084308990844D44908440544B5
:103C1000A80540EA9525354405EA060027EA05018E
:103C2000084309990844CE4908440444E00140EAA5
:103C300054642C4404EA050026EA040108430A9966
:103C40000844C84908440744380340EA1757274442
:103C500007EA040025EA070108430B990844A0F588
:103C600024404F380644700440EAD6363E4406EA03
:103C7000070024EA060108430C990844BA4908449D
:103C80000544A80540EA9525354405EA060027EADB
:103C9000050108430D990844B44908440444E0016F
:103CA00040EA54642C4404EA050026EA040108436F
:103CB0000E990844AE4908440744380340EA1757B0
:103CC000274407EA040025EA070108430F9908443E
:103CD000A84908440644700440EAD6363E4406EA41
:103CE000070024EA0601084310990844A249084441
:103CF0000544A80540EA9525354405EA070026EA6B
:103D000007010843029908449C490844044460019F
:103D100040EAD4642C4404EA060025EA060108437C
:103D200007990844964908440744780240EAD7575F
:103D3000274407EA050024EA050108430C990844D2
:103D4000904908440644B00340EA96463E4406EAD9
:103D5000040027EA04010843019908448A490844F9
:103D60000544280540EA1535354405EA070026EAEA
:103D70000701084306990844844908440444600143
:103D800040EAD4642C4404EA060025EA060108430C
:103D90000B9908447E4908440744780240EAD75703
:103DA000274407EA050024EA05010843109908445E
:103DB000784908440644B00340EA96463E4406EA81
:103DC000040027EA0401084305990844724908449D
:103DD0000544280540EA1535354405EA070026EA7A
:103DE000070108430A9908446C49084404446001E7
:103DF00040EAD4642C4404EA060025EA060108439C
:103E00000F990844664908440744780240EAD757A6
:103E1000274407EA050024EA0501084304990844F9
:103E2000604908440644B00340EA96463E4406EA28
:103E3000040027EA04010843099908445A49084440
:103E40000544280540EA1535354405EA070026EA09
:103E5000070108430E99084454490844044460018A
:103E600040EAD4642C4404EA060025EA060108432B
:103E7000039908444E4908440744780240EAD7575A
:103E8000274407EA050024EA050108430899084485
:103E9000484908440644B00340EA96463E4406EAD0
:103EA000040027EA040108430D99084442490844E4
:103EB0000544280540EA1535354485EA0600784072
:103EC000069908443D4908440444200140EA14741A
:103ED0002C4484EA05007040099908443849084494
:103EE0000744F80240EA5757274487EA040068402D
:103EF0000C990844334908440644300440EA164605
:103F00003E4486EA070060400F9908442E49084461
:103F10000544E80540EA5525354485EA0600784021
:103F200002990844294908440444200140EA1474D1
:103F30002C4484EA0500704005990844244949E06E
:103F400078A46AD756B7C7E8DB702024EECEBDC18F
:103F5000AF0F7CF52AC68747134630A8019546FD6A
:103F6000D8988069AFF7448BBED75C892211906BDB
:103F7000937198FD8E4379A62108B44962251EF6F7
:103F800040B340C0515A5E26AAC7B6E95D102FD68D
:103F90005314440281E6A1D8C8FBD3E7E6CDE12162
:103FA000D60737C3870DD5F4ED145A4505E9E3A9C3
:103FB000F8A3EFFCD9026F678A4C2A8D4239FAFFC9
:103FC00081F6718722619D6D0C38E5FD44EABEA43F
:103FD000A9CFDE4B08440744F80240EA575727446C
:103FE00087EA0400684008990844A7490844064441
:103FF000300440EA16463E4486EA070060400B99CA
:104000000844A24908440544E80540EA55253544DA
:1040100085EA060078400E9908449D490844044406
:10402000200140EA14742C4484EA05007040019990
:104030000844984908440744F80240EA575727447F
:1040400087EA0400684004990844934908440644F8
:10405000300440EA16463E4486EA0700604007996D
:1040600008448E4908440544E80540EA552535448E
:1040700085EA060078400A990844894908440444BE
:10408000200140EA14742C4484EA050070400D9924
:104090000844844908440744F80240EA5757274433
:1040A00087EA04006840109908447F4908440644A0
:1040B000300440EA16463E4486EA07006040039911
:1040C00008447A4908440544E80540EA5525354442
:1040D00065EA0700704001990844754908440444A2
:1040E000A00140EA94642C4464EA06006840089900
:1040F0000844704908440744B80240EA97572744E7
:1041000067EA050060400F9908446B49084406447B
:10411000F00340EA56463E4466EA040078400699B9
:104120000844664908440544680540EAD5253544F5
:1041300065EA070070400D99084461490844044449
:10414000A00140EA94642C4464EA060068400499A3
:1041500008445C4908440744B80240EA975727449A
:1041600067EA050060400B99084457490844064433
:10417000F00340EA56463E4466EA0400784002995D
:104180000844524908440544680540EAD5253544A9
:1041900065EA07007040099908444D490844044401
:1041A000A00140EA94642C4464EA06006840109937
:1041B0000844484908440744B80240EA975727444E
:1041C00067EA0500604007990844434908440644EB
:1041D000F00340EA56463E4466EA040078400E99F1
:1041E00008443E4908440544680540EAD52535445D
:1041F00065EA0700704005990844394908440444B9
:10420000A00140EA94642C4464EA060068400C99DA
:104210000844344908440744B80240EA9757274401
:1042200067EA05006040039908442F4908440644A2
:10423000F00340EA56463E4466EA040078400A9994
:1042400008442A4908440544680540EAD525354410
:10425000D8F800002044C8F80000D8F8040028442A
:10426000C8F80400D8F808003044C8F80800D8F8A6
:104270000C003844C8F80C004022002101A800F0CE
:1042800083F811B0BDE8F083604BBBF670BCBFBED5
:10429000C67E9B28FA27A1EA8530EFD4051D880445
:1042A00039D0D4D9E599DBE6F87CA21F6556ACC4B9
:1042B000442229F497FF2A43A72394AB39A093FC07
:1042C000C3595B6592CC0C8F7DF4EFFFD15D848583
:1042D0004F7EA86FE0E62CFE144301A3A111084E07
:1042E000827E53F735F23ABDBBD2D72A91D386EB03
:1042F0002DE9F047044688461546208AC0F3C509D3
:10430000206900EBC5002061B0EBC50F02D26069E7
:10431000401C6061606900EB55716161C9F1400743
:10432000BD421BD304F1180101EB09003A46414696
:1043300000F020F804F118012046FFF7EBFB3E46A1
:1043400005E008EB06012046FFF7E4FB403606F1E6
:104350003F00A842F5D34FF0000900E00026AA1B59
:1043600008EB060104F1180303EB090000F002F862
:10437000BDE8F08710B50346002002E00C5C1C5439
:10438000401C9042FAD310BD10B50346002001E056
:104390001954401C9042FBD310BD00000EB5002004
:1043A0000090019002901E481E49086081151D482A
:1043B0008160002101730121017581614FF4602149
:1043C000C161002017494860032116480161FCF7CC
:1043D000F3FE08B1FCF7CFFB0A200090012001900A
:1043E0000720029069460F48FCF7A8FD08B1FCF7CA
:1043F000C2FB0B2000900220019069460948FCF79F
:104400009DFD08B1FCF7B7FB0C2000900320019044
:1044100069460448FCF792FD08B1FCF7ACFB0EBD01
:10442000002401404C0F002008B500BF124840692D
:1044300040F00100104948610846406900F0010061
:10444000009000BF00BF002205210D20FDF7E0FF16
:104450000D20FDF7CDFF002205210E20FDF7D8FF2E
:104460000E20FDF7C5FF002205210F20FDF7D0FF2C
:104470000F20FDF7BDFF08BD0010024000B59DB044
:104480001C22184916A8FBF7D1FE002116A802F03D
:104490006CFB154908601C2212491C310FA8FBF760
:1044A000C5FE00210FA802F060FB104908601C2225
:1044B0000C49383108A8FBF7B9FE002108A802F022
:1044C00054FB0B4908601C220649543101A8FBF734
:1044D000ADFE002101A802F048FB064908601DB0AE
:1044E00000BD0000B47F00085C00002060000020D8
:1044F000640000206800002000B585B00020019015
:1045000002900390049000BF3A48806940F0100088
:10451000384988610846806900F01000009000BFAB
:1045200000BF00BF0846806940F02000886108464F
:10453000806900F02000009000BF00BF00BF084667
:10454000806940F0040088610846806900F004003A
:10455000009000BF00BF00BF0846806940F008001F
:1045600088610846806900F00800009000BF00BF25
:10457000002241F279012048FDF784FE4FF6F870E1
:1045800001900320029001A91C48FDF7C9FCFF20FF
:10459000019000200290039001A91948FDF7C0FC8A
:1045A00041F2790001900120029000200390022046
:1045B000049001A91048FDF7B3FC4EF2863001903B
:1045C0000320029001A90C48FDF7AAFC4FF4194002
:1045D00001900320029001A90948FDF7A1FC0420E5
:1045E00001900320029001A90648FDF799FC05B04F
:1045F00000BD000000100240000C0140001001400E
:10460000000801400014014000B587B0002003906D
:10461000049005900690019002904FF0804015495B
:10462000086040F21F30486000211248816041F666
:104630003F71C1600021016180218161FEF748FC6A
:1046400008B1FCF798FA4FF48050039003A9094889
:10465000FEF7DAFC08B1FCF78EFA00200190029018
:1046600001A90448FEF7E6FB08B1FCF784FA07B09D
:1046700000BD0000B80F002010B50B480B490860C2
:104680004FF416504860002108488160C160016104
:104690000C21416100218161C161FFF731F808B14E
:1046A000FCF769FA10BD00000038014030470020D7
:1046B00010B50B480B4908604FF4165048600021B4
:1046C00008488160C16001610C2141610021816164
:1046D000C161FFF715F808B1FCF74DFA10BD0000F5
:1046E000004800407847002000BFFEE710B586B0C4
:1046F000FE480078012831D10621FD4801F016FF5F
:10470000FB498979FA4AD27941EA02218842F2D1F9
:10471000F84800880A2821DAF5480078F64909782F
:1047200088421CD1F2484078032818D1F04880789C
:10473000A8B9EF48C078012811D1ED48007970B9C7
:10474000EB48407901280AD107200090EB48037814
:1047500002220321E848008802F058FE91E3E44871
:104760000078E549097888421CD1E148407803285F
:1047700018D1DF488078A8B9DD48C078022811D167
:10478000DB48007970B9DA48407901280AD107205E
:104790000090DB48037802220321D748008802F00A
:1047A00035FE6EE3D2480078D349097888421CD19F
:1047B000CF484078032818D1CD488078A8B9CC4894
:1047C000C078032811D1CA48007970B9C848407927
:1047D00001280AD107200090CA4803880222032139
:1047E000C548008802F012FE4BE3C1480078C24978
:1047F000097888421CD1BE484078032818D1BC48AB
:104800008078A8B9BA48C078042811D1B84800798E
:1048100070B9B748407901280AD107200090BA48FA
:10482000038802220321B448008802F0EFFD28E348
:10483000AF480078B049097888421CD1AC4840782C
:10484000032818D1AA488078A8B9A948C0780528B3
:1048500011D1A748007970B9A548407901280AD13B
:1048600007200090A948038802220321A24800885B
:1048700002F0CCFD05E39E4800789F490978884204
:104880001FD19B48407803281BD199488078C0B934
:104890009748C078012814D19548007988B9944880
:1048A000407902280DD1092095490978CDE90010F9
:1048B00092480378042203218F48008802F010FEFA
:1048C000DFE28B4800788C490978884222D18848F9
:1048D000407803281ED186488078D8B98448C078AB
:1048E000012817D182480079A0B98148407903286E
:1048F00010D10B2183480088814A1278CDE900202D
:1049000002917E480378062203217B48008802F04A
:1049100085FCB6E27648007877490978884225D147
:1049200073484078032821D171488078F0B97048E5
:10493000C07801281AD16E480079B8B96C4840791E
:10494000042813D10D22704800886E4909886C4BE9
:104950001B78CDE90031CDE90202684803780822CE
:1049600003216548008802F0A1FC8AE260480078D3
:1049700061490978884228D15D484078032824D1CC
:104980005B48807808BB5A48C07801281DD1584838
:104990000079D0B956484079052816D10F215B48D7
:1049A000028859480088574B1B88CDE90130CDE972
:1049B0000321534800780090504803780A220321CD
:1049C0004D48008802F0C6FC5BE2494800784A493D
:1049D000097888421FD14648407803281BD14448B3
:1049E0008078C0B94248C078022814D14048007984
:1049F00088B93F48407902280DD1092041490988EA
:104A0000CDE900103E480378042203213A4800888B
:104A100002F066FD35E23648007837490978884269
:104A200022D13348407803281ED131488078D8B944
:104A30002F48C078022817D12D480079A0B92C48FA
:104A40004079032810D10B212F4800882D4A128865
:104A5000CDE9002002912A48037806220321264846
:104A6000008802F0DBFB0CE221480078224909783B
:104A7000884225D11E484078032821D11C488078DF
:104A8000F0B91B48C07802281AD119480079B8B982
:104A900017484079042813D10D211C4800881A4A70
:104AA0001288184B1B88CDE90032CDE90201144869
:104AB0000378082203211048008802F0F7FBE0E1A8
:104AC0000B4800780C490978884232D10848407870
:104AD00003282ED10648807858BB0548C0780328A3
:104AE00027D10348007920BB014811E01D050020B3
:104AF000843A00201E0500204E00002058000020AF
:104B00005900002072000020740000207000002076
:104B1000407902280DD10920DB490988CDE9001030
:104B2000DA48038804220321D948008802F0D8FC1F
:104B3000A7E1D8480078D6490978884222D1D548DB
:104B4000407803281ED1D3488078D8B9D148C0789E
:104B5000032817D1CF480079A0B9CE48407903285F
:104B600010D10B21CC480088C74A1288CDE900201B
:104B70000291C648038806220321C548008802F036
:104B80004DFB7EE1C3480078C149097888421FD1B6
:104B9000C048407803281BD1BE488078C0B9BD48C2
:104BA000C078042814D1BB48007988B9B948407945
:104BB00002280DD10920B8490988CDE90010B24872
:104BC000038804220321B248008802F089FC58E1DE
:104BD000B0480078FA281BD1AE484078032817D196
:104BE000AC488078A0B9AB48C078AA2810D1A948B1
:104BF000007968B9A7484079012809D107200090B9
:104C0000A348038802220321FA2002F0FFFB38E1C7
:104C1000A04800789E490978884224D19D48407870
:104C2000032820D19B48807850281CD19948C0780F
:104C3000C8B998480079B0B996484079022812D18D
:104C400009219648008880B2CDE9000193480068A8
:104C50004FF6FF7101EA1043042203218C480088BB
:104C600002F03EFC0DE18B480078894909788842C2
:104C700029D188484078062825D18648807810BBFD
:104C80008448C07802281ED182480079D8B9814969
:104C9000487902F09FFC05227E49814801F096F98F
:104CA0007C4840797B4C247940EA04237948C078D9
:104CB000784CA47840EA0422764841787448008809
:104CC00002F0DAFBDDE07348007871490978884228
:104CD00029D170484078062825D16E48807810BBCD
:104CE0006C48C0780A281ED16A480079D8B969484A
:104CF0004079012817D1002266496A4801F066F917
:104D000064484079634C247940EA04236148C078C0
:104D1000604CA47840EA04225E4841785C480088F0
:104D200002F0AAFBADE05B48007859490978884257
:104D300029D158484078062825D15648807810BB9C
:104D40005448C0780B281ED152480079D8B9514830
:104D50004079012817D100224E49534801F036F915
:104D60004C4840794B4C247940EA04234948C078A8
:104D7000484CA47840EA04224648417844480088D8
:104D800002F07AFB7DE04348007841490978884287
:104D900029D140484078062825D13E48807810BB6C
:104DA0003C48C0780C281ED13A480079D8B9394916
:104DB000487902F045FC052236493C4801F006F9E5
:104DC00034484079334C247940EA04233148C07890
:104DD000304CA47840EA04222E4841782C480088C0
:104DE00002F04AFB4DE02B480078294909788842B7
:104DF00025D128484078062821D126488078F0B966
:104E00002448C078AA281AD122480079B8B90522C6
:104E10002049274801F0DAF81E4840791D4C2479D2
:104E200040EA04231B48C0781A4CA47840EA0422C4
:104E3000184841781648008802F01EFB21E015480A
:104E4000007813490978884217D11248407806281B
:104E500013D11048807880B90E48C078CC280CD186
:104E60000C480079A52808D10A4840795A2804D16D
:104E700001F094FBFDF71EFB03E001F08FFB02F055
:104E80008FF906B010BD00007400002072000020F1
:104E90004E000020843A00207000002054000020C2
:104EA0000008070800180708002007080010070876
:104EB0000000070800BFFEE7FEB50020F9490870B2
:104EC000F948407AF849097A40EA0120F749088010
:104ED000F7480588F7A103C9CDE90101F248C07977
:104EE000F64908704FF48061F548FBF7B8F94FF4C4
:104EF0008061F448FBF7B3F9F0480078012804D04A
:104F000002287DD004287CD1ADE12822E6490A316F
:104F1000ED48FBF78BF98021E3480A3001F076FB7E
:104F2000EA490880E81EE049095C281FDE4A105C57
:104F300041EA0020E6490880E44800880988884260
:104F40007ED100240AE0E3482044017904F10A00FC
:104F5000D54A105C814200D002E0641C582CF2DB80
:104F600000BF322C6DDA00240FE00A2000EB440071
:104F7000CD49085C0B2101EB4401CB4A515C40EA6E
:104F80000120CF4921F81400641C192CEDDB1922F3
:104F9000D049091DCA48FBF7B9FE322001F057FB82
:104FA0000120CD490860CB491B31CC4802F008F9FB
:104FB000C948006830B3C948007800F00F0042F2D9
:104FC00010714843C549497801F00F0101EB4102D6
:104FD000C2EBC11100EBC101C048807800F00F00A6
:104FE00000EBC00202EB001001EB8000BB49C97866
:104FF00001F00F0101EB810100EB4100B74902E034
:10500000BBE0DFE106E0097901F00F010844B44993
:10501000086022E0B148007800F00F004FF47A7188
:105020004843AE49497801F00F0101EBC10202EBA0
:10503000011100EB8100A949897801F00F0101E01D
:1050400081E061E001EB810100EB4101A348C07800
:1050500000F00F000844A2490860A1480068A14977
:105060000860A14801F0FCFAFCF742FF9D480023CC
:105070009D4902680120FCF7E3FEFCF7D7FE964845
:105080000068F8B11022934921319848FBF728FEB7
:10509000082297499548FBF739FE00200FE0934915
:1050A00031F810104FF47F4202EA01218F4A32F8A2
:1050B000102041EA12218D4A22F81010401C0828C5
:1050C000EDDB1EE01022834920318848FBF708FE03
:1050D000082287498548FBF719FE00200FE0834925
:1050E00031F810104FF47F4202EA01217F4A32F872
:1050F000102041EA12217D4A22F81010401C082895
:10510000EDDB7C487C4908604FF480616648FBF722
:10511000A6F8502001F09BFA7848807900907748F3
:105120004079764E367940EA06237448C078734E4B
:10513000B67840EA0622714841787148008802F04A
:105140000FFA00BF0EE04FF480615748FBF787F875
:1051500001A8FBF78FF886B26423324601A969489B
:10516000FEF709FC4FF480615548FBF778F84FF4DF
:1051700080615448FBF773F825E180214A480A30E2
:1051800001F044FA51490880E81E4749095C281F8C
:10519000454A105C01EB00204D4908804B480088CF
:1051A000098888425ED100240FE00A2000EB440009
:1051B0003D49085C0B2101EB44013B4A515C40EA4C
:1051C00001203F4921F81400641C402CEDDB4022F3
:1051D000494801683A48FBF799FD47480068803024
:1051E00045490860012211464748FDF74BF8012068
:1051F000FCF7B0FD002201214348FDF743F82A489F
:10520000C0782949897840EA01203B49098889B258
:1052100088420AD001A8FBF72DF886B264233246F3
:1052200001A93848FEF7A7FBCDE04FF480611E4886
:10523000FBF715F8502001F00AFA30488079009009
:105240002E4840792D4E367940EA06232B48C07807
:105250002A4EB67840EA0622284841782848008835
:1052600002F07EF9AFE080210F480A3001F0CEF95C
:1052700016490880E81E0C49095C281F0A4A105C80
:1052800001EB0020124908801048008809888842F4
:105290006FD108220F490E311C48FBF721FD002079
:1052A00046E000001C05002084320020120000208F
:1052B0001E0500206572726F720D0A00000000204A
:1052C00082060020820A002010060020180000201C
:1052D0001A0000207AF007082C0000205806002051
:1052E000200000203000002000480708720600203F
:1052F00000500708000006081C000020843A002027
:105300004E00002030470020000C01400200002029
:105310002E4931F810104FF47F4202EA01212B4A46
:1053200032F8102041EA1221284A22F81010401CBD
:105330000428EDDB2649254801F04AF9254801F00B
:105340008FF9FCF7D5FD224800232249026802208C
:10535000FCF776FDFCF76AFD1F4801681F48FBF764
:10536000FBFA1F4908600846006818B100F082F88F
:1053700027E016E01BA11F4800F0D2FE0646502091
:1053800001F065F9B2B21B491B48FEF74DFB02E084
:105390000120FCF7DFFC184890F841002128F7D0E5
:1053A0000FE0502001F053F901A8FAF763FF86B22D
:1053B0006423324601A91048FEF7DDFA502001F0BF
:1053C00046F900E000BF00BFFEBD00000200002063
:1053D00054000020004007083000002000000608AC
:1053E00028000020636865636B3D6572726F720D03
:1053F0000A000000843200203047002008B5084928
:105400000968C9084FF47A72B1FBF2F14143009187
:1054100000BF00BF00994A1E00920029F9D108BDC3
:10542000A405002070B504460D4629462046FCF729
:1054300017FF08B9012070BD0020FCE708B50A4835
:105440000A4908600846008880B2ADF802000846A4
:105450000068000CADF80000022205496846FBF721
:1054600055FC00F08DFE0000BBBB5555240000200C
:105470007AF0070808B54FF0AA30154908600846C9
:10548000008880B2ADF800000846008880B2ADF810
:10549000020008460068009004220E496846FBF7A7
:1054A00035FC0DA10F4800F03BFE0446A2B20D49A9
:1054B0000D48FEF7B9FA02E00120FCF74BFC0A4860
:1054C00090F841002128F7D000BF00BF00F058FE3F
:1054D000240000207AF007087265626F6F740D0A6D
:1054E00000000000843200203047002000BF01206F
:1054F00001F02AFB012211460B48FCF7C3FE0120F4
:10550000FCF728FC002201210748FCF7BBFEFBF753
:10551000DFFC06490870FBF707FD054908700548E0
:10552000FBF738FCE3E70000000C014058000020C6
:10553000590000204C0F002000BF012001F004FBA7
:10554000FBE700BF012001F0FFFAFBE7F0B587B0F1
:1055500002225E4906A8FBF7C3FBBDF81A00BDF89E
:10556000181040EA01405A4908605A4800685A49F0
:1055700008604FF480615948FAF771FE5648006898
:1055800000F50060C0F3CF2651480068B0F1AA3F93
:1055900012D0B0F1FF3F04D051490844002874D123
:1055A00074E050A14D4800F0BBFD0446A2B24B4947
:1055B0004F48FEF739FA85E0002002904D480490EC
:1055C000059600200190FCF793FC01A902A8FCF7C6
:1055D000D5FB0746FCF72AFC3E4800683E490860B8
:1055E000084601684448FBF7B7F90546CDB13A488B
:1055F000414902683F4801F099F940A1374800F05D
:105600008FFD0446A2B235493948FEF70DFA02E093
:105610000120FCF79FFB364890F841002128F7D085
:1056200017E039A12D4800F07BFD0446502001F021
:105630000EF8A2B229492E48FEF7F6F902E0012041
:10564000FCF788FB2A4890F841002128F7D007B0E2
:10565000F0BD214801682748FBF77EF9A0B12DA1D4
:105660001E4800F05DFD0446A2B21C492048FEF72A
:10567000DBF902E00120FCF76DFB1D4890F84100CA
:105680002128F7D0FFF7DAFE1CE01AE024A1134826
:1056900000F046FD0446A2B210491548FEF7C4F9D1
:1056A00002E00120FCF756FB114890F84100212848
:1056B000F7D0002080F3138800BF0E48FEF7DAF918
:1056C00000E0C4E700BF00BFC1E700007AF00708B0
:1056D000380000202000002030000020843200200C
:1056E0004544AAAA6E6F726D616C53746172740046
:1056F000304700200000040800000608757064614F
:1057000074650D0A00000000636865636B6661697B
:105710006C0000007570646174656F6B0D0A0000A9
:105720006A756D700000000000BF012001F00CFAE6
:105730001248007801281ED1114800888E281AD1FD
:105740001048007810490978884214D10D484078F3
:10575000102810D18C210D4800F0E8FE094991F87D
:105760008C10084A92F88D2041EA0221884202D129
:10577000FFF7A2FBD9E7FEF7B9FFD6E71C0500202B
:105780001E050020843A00204E00002084320020B4
:1057900010B500BF502080F31188BFF34F8FBFF3C7
:1057A0006F8F00BF02F0C0FA18B14FF0805004496B
:1057B000086000BF002080F3118800BF10BD00000A
:1057C00004ED00E000B595B028210BA8FAF747FDDD
:1057D000142106A8FAF743FD18216846FAF73FFDA1
:1057E00001200B9000040C9000200D9001200F90E0
:1057F00002201290C1031391002114910BA8FDF710
:10580000E5F808B1FBF7B7F90F20069002200790E2
:1058100080200890C000099000200A90002106A86E
:10582000FCF78EFF08B1FBF7A6F9022000904003B9
:1058300002906846FCF7ECFE08B1FBF79CF915B046
:1058400000BD704710B54FF480510348FCF710FDC0
:105850000248FDF760FC10BD000C0140B80F0020AD
:1058600010B50248FDF757FC10BD00008C48002021
:1058700010B50268204B98420ED0204B98420BD0B6
:10588000B0F1804F08D01E4B984205D01D4B984276
:1058900002D01D4B984203D122F070024B681A438C
:1058A000154B98420ED0154B98420BD0B0F1804F5B
:1058B00008D0134B984205D0124B984202D0124B9D
:1058C000984203D122F44072CB681A4322F080033D
:1058D0004C6943EA040202608B68C3620B6883620E
:1058E000054B984202D0054B984201D10B690363E6
:1058F0000123436110BD0000002C01400034014031
:105900000004004000080040000C004030B50C4688
:10591000816821F47F4142EA0325254329438160C0
:1059200030BD0A46816821F0700142F00703194337
:105930008160704730B50B461446026A056A25F04F
:1059400001050562816921F0F00141EA041122F0AC
:105950000A021A438161026230BD30B50B4614461B
:10596000026A056A25F010050562816921F470411B
:1059700041EA043122F0A00242EA0312816102628C
:1059800030BD70B505466C6A0020E085E084204695
:10599000FDF742FD70BD70B506460025746A2068AB
:1059A0004069C0F3C01594F84100212805D125B104
:1059B0000020E084204600F0C8F820684069C0F369
:1059C000801594F84200222805D125B10020E085F9
:1059D000204600F074F8606C40F0100060642046CF
:1059E000FDF71AFD70BD70B505466C6A2868006841
:1059F00000F02000002842D1E08500BF00BF2168F0
:105A00000C3151E8001F21F4807021680C3141E80D
:105A10000002002AF3D100BF00BF00BF216814318B
:105A200051E8001F21F001002168143141E8000213
:105A3000002AF3D100BF00BF00BF2168143151E834
:105A4000001F21F040002168143141E80002002AC3
:105A5000F3D100BF202084F84200206B01280ED132
:105A600000BF00BF21680C3151E8001F21F0100079
:105A700021680C3141E80002002AF3D100BF002068
:105A80006063206B012804D1A18D2046FDF71DFC29
:105A900002E02046FDF766FF70BD70B505466C6AF2
:105AA00001206063206B012805D1A08D41082046AC
:105AB000FDF70BFC02E02046FDF75CFF70BD00BF68
:105AC00000BF02680C3252E8002F22F49071026885
:105AD0000C3242E80013002BF3D100BF00BF00BF1F
:105AE0000268143252E8002F22F0010102681432D9
:105AF00042E80013002BF3D100BF016B01290ED146
:105B000000BF00BF02680C3252E8002F22F01001E3
:105B100002680C3242E80013002BF3D100BF2021B1
:105B200080F8421000210163704710B504462068D8
:105B3000C06820F040002168C860202084F841003F
:105B40002046FDF78DFF002010BD00BF00BF02689A
:105B50000C3252E8002F22F0C00102680C3242E8F9
:105B60000013002BF3D100BF202180F841107047B3
:105B7000F8B5044694F84200222875D1A068B0F523
:105B8000805F0CD1206950B90025A66A2068406862
:105B9000C0F308003080A06A801CA06215E0A56AEE
:105BA0000026A068B0F5805F03D0A06828B92069FE
:105BB00018B920684068287004E02068406800F048
:105BC0007F002870A06A401CA062E08D401E80B259
:105BD000E085002846D12068C06820F020002168B8
:105BE000C8602068C06820F480702168C8602068A0
:105BF000406920F0010021684861202084F84200BB
:105C000000206063206B012826D10020206300BFA4
:105C100000BF21680C3151E8001F21F010002168FD
:105C20000C3141E80002002AF3D100BF206800686F
:105C300000F0100010280AD100BF0020009020685A
:105C40000068009020684068009000BF00BFA18DF0
:105C50002046FDF73AFB02E02046FDF783FE0020D8
:105C6000F8BD01E00020FBE70220F9E770B504462B
:105C70002168096921F44051E268114322681161E9
:105C80002269A1681143626941EA02052168C96875
:105C900041F20C62914329432268D160216849692D
:105CA00021F44071A2691143226851612D4A216893
:105CB000914202D1FCF742FE01E0FCF72FFE00EB1F
:105CC000C00101EB001162689200B1FBF2F100EB40
:105CD000C00202EB001263689B00B2FBF3F2642384
:105CE000B2FBF3F202EBC20303EB0212A1EB82015F
:105CF000322202EB01116422B1FBF2F101F0F0015A
:105D000000EBC00202EB001263689B00B2FBF3F2EF
:105D10006423B2FBF3F201EB021200EBC00101EBD2
:105D2000001163689B00B1FBF3F100EBC00303EBD0
:105D300000136668B600B3FBF6F36426B3FBF6F314
:105D400003EBC30606EB0313A1EB8301322303EB42
:105D500001116423B1FBF3F101F00F01114422683A
:105D6000916070BD0038014077B581B0044615469A
:105D70000298A062A58500206064222084F8420079
:105D80002848E16B88622848E16BC8622748E16BCC
:105D900008630020E16B486302AE32682368191D76
:105DA0002B46E06BFBF788FF00BF002000902068C7
:105DB0000068009020684068009000BF00BF206924
:105DC00070B100BF00BF21680C3151E8001F41F4E1
:105DD000807021680C3141E80002002AF3D100BF35
:105DE00000BF00BF2168143151E8001F41F00100DD
:105DF0002168143141E80002002AF3D100BF00BF3E
:105E000000BF2168143151E8001F41F040002168B3
:105E1000143141E80002002AF3D100BF002004B091
:105E200070BD0000E75900089B5A00089759000808
:105E3000014691F84100212828D18868B0F5805F9B
:105E40000BD1086948B90A6A1088C0F308000B68CA
:105E50005860086A801C086205E00B6A581C0862DA
:105E600018780B685860C88C401E80B2C88458B936
:105E70000868C06820F080000B68D8600868C068B7
:105E800040F040000B68D860002070470220FCE71B
:105E90002DE9F04104460D4617469846069E34E02B
:105EA000701C88B32EB1FCF7F3F9A0EB0800B042E8
:105EB0002BD900BF00BF21680C3151E8001F21F42D
:105EC000D07021680C3141E80002002AF3D100BFF4
:105ED00000BF00BF2168143151E8001F21F001000C
:105EE0002168143141E80002002AF3D100BF2020CC
:105EF00084F8410084F8420000BF002084F840008C
:105F000000BF0320BDE8F081FFE72068006828405B
:105F1000A84201D1012000E00020B842C0D00020FA
:105F2000F0E7000008B51C4800680068C0F30010E6
:105F300068B300BF00200090174800680068009018
:105F4000154800684068009000BF00BF1248FDF788
:105F50001EFA124800684068C0F580601049088049
:105F6000084602880F491048FAF760F90C48028881
:105F70000C490E48FAF75AF94FF48062094906486D
:105F8000FDF7DAFC01200A4908700A490870024846
:105F9000FDF744FA08BD000030470020C04700204C
:105FA0001E0500208436002084320020843A002020
:105FB0001C0500201D05002010B50248FDF72EFA33
:105FC00010BD00007847002000BFFEE72DE9F04734
:105FD00005460F4690460024284600F041FBFBF79B
:105FE00087FF414885420CD117F80840224600231C
:105FF00001460120FBF724FF06460EB93B4804800A
:106000006EE03B4885420CD117F808402246002339
:1060100001460120FBF714FF06460EB935490C7006
:106020005EE0354885420CD117F80840224600232F
:1060300001460120FBF704FF06460EB92F480480F5
:106040004EE02F48854202D02E48854248D14FF479
:106050003A762B4885421FD12B480088B04204DB9A
:1060600029480088801B84B205E027480088301A40
:1060700084B244F400442246002321490120FBF766
:10608000DFFE8146B9F1000F05D1C4F30E001F49B0
:1060900008801F48048022E01A4885421FD11D480D
:1060A0000088B04204DB1B480088801B84B205E0F6
:1060B00018480088301A84B244F400442246002371
:1060C00010490120FBF7BCFE8146B9F1000F05D154
:1060D000C4F30E00104908801048048000BF00BFC0
:1060E000FBF7A4FEBDE8F087000007084E00002083
:1060F0000008070859000020001007085000002081
:1061000000180708002007087A0000207E00002001
:106110006C0000207C000020800000206E00002029
:106120000FB4084B10B504A902AA039800F058F860
:10613000044602A9002000F0F4F9204610BC5DF8E6
:1061400014FB00002365000802480068C0F3022029
:10615000704700000CED00E010B5002804DB0A07D2
:10616000130E054A135406E00A07140E034A00F002
:106170000F031B1FD45410BD00E400E018ED00E035
:1061800000BF00BF00BFBFF34F8F00BF00BF00BF05
:106190000948006800F4E06008490843001D06490A
:1061A000086000BF00BF00BFBFF34F8F00BF00BF3C
:1061B00000BF00BF00BFFDE70CED00E00000FA05E6
:1061C00002E008C8121F08C1002AFAD170477047C0
:1061D000002001E001C1121F002AFBD1704700001E
:1061E0002DE9FF4F8BB088460546002606E025289E
:1061F0000BD0DDE90D1290476D1C761C2878002825
:10620000F5D10FB03046BDE8F08F0024A146A2467C
:106210000122AE4900E0044315F8013F203B02FA99
:1062200003F00842F7D128782A2810D06FF02F0207
:106230002878A0F13001092915D809EB890102EB72
:10624000410144F0020400EB01096D1CF0E758F82D
:10625000041B5FEA010903D544F40054C9F10009A5
:1062600044F002046D1C28782E2817D115F8010F70
:1062700044F004042A280ED06FF02F022878A0F1F1
:10628000300109290AD80AEB8A0102EB410100EB2F
:10629000010A6D1CF2E758F804AB6D1C28786C28D5
:1062A0000FD006DC4C2817D068280DD06A2814D1EE
:1062B00004E0742810D07A280FD10DE044F40014C3
:1062C0000AE044F4801401E044F440146978814207
:1062D00002D104F580146D1C6D1C2878692865D0E6
:1062E00006DC00288DD0632827D0642806D15DE025
:1062F0006E2808D073282AD0752877D0DDE90D12D2
:106300009047761CE0E0C4F30250022809D003282D
:106310000DD0D8F8001004280DD00E6008F1040844
:10632000D2E0D8F80010F217C1E90062F6E7D8F819
:1063300000100E80F2E70E70F0E718F8041B8DF8DD
:10634000001000208DF80100EB46012003E058F812
:1063500004BB4FF0FF3061074FF0000701D40AE0A3
:106360007F1C57450DDA8742FADB1BF8071000291E
:10637000F6D106E07F1C8742FCDB1BF807100029E2
:10638000F8D1DDE90D23A9EB07008146214600F095
:10639000B1F83044C61904E0DDE90D121BF8010B19
:1063A00090477F1EF8D22146484688E058F8040BF3
:1063B000C4F302514FF00A0B032900D100B20429A3
:1063C00000D140B2002802DA40422D2102E021052E
:1063D00005D52B218DF82410012104E006E0E1070A
:1063E00010D02021F6E708AF089113E058F8040B0D
:1063F000C4F302514FF00A0B032900D180B20429E3
:1064000000D1C0B20021EEE75946FAF7F3F8303177
:1064100007F8011D0028F7D1ADEB070000F1200BB4
:10642000600702D524F4803401E04FF0010ADA4518
:1064300002DDAAEB0B0000E00020824600EB0B011E
:1064400008980144A9EB01000A90E00306D4DDE9B5
:106450000D2321460A9800F04DF806444FF000093C
:1064600008E009A911F80900DDE90D12904709F1CA
:106470000109761C08998945F3DBE0030CD5DDE9B9
:106480000D2321460A9800F035F8064404E0DDE9C2
:106490000D1230209047761CBAF10001AAF1010AD2
:1064A000F5DC05E0DDE90D1217F8010B9047761CCD
:1064B000BBF10001ABF1010BF4DC0A982146DDE9E8
:1064C0000D2300F005F806446D1C97E6092801002D
:1064D0002DE9F041044600251E461746880404D4E1
:1064E00005E039462020B0476D1C641EF9D52846CA
:1064F000BDE8F0812DE9F041044600251E46904696
:10650000C80301D5302700E02027880404D505E022
:1065100041463846B0476D1C641EF9D52846BDE893
:10652000F0810A68531C0B601070704730B502464A
:106530000B464FF6FF70002110E0545C60400024D1
:1065400009E000F0010525B14AF2010585EA600085
:1065500000E04010641C082CF3DB491C9942ECDB82
:1065600030BD000010B504460B480068C06820F438
:10657000005009490968C86007484460FDF7C0F841
:1065800008B1FAF7F8FA04480068C06840F400500F
:1065900001490968C86010BD3047002010B54FF4AC
:1065A00080610748F9F75BFE4FF480610548F9F711
:1065B00056FE0020044908700449087010BD000010
:1065C000843A0020843600201D0500201C05002090
:1065D00010B50288C2F30323027863F31F12130677
:1065E0004288C2F3032464F31F1243EA0243828801
:1065F000C2F3032464F31F1243EA0223C288C2F3E6
:10660000032464F31F1213430B6010BD30B5024620
:106610000B460020002117E0545C80EA042000248F
:106620000EE000F400452DB141F2210585EA400558
:10663000A8B203E04FF6FF7505EA4000651CECB216
:10664000082CEEDB4C1CA1B29942E5DB30BDC20048
:10665000002100BF01E000BF491C9142FBD37047FD
:1066600030B585B0044600200190039401200490C9
:1066700000200090FBF73CFC694601A8FBF77EFB7D
:106680000546FBF7D3FB15BB1248844203D100201B
:10669000114908801BE01148844203D100201049B1
:1066A000087014E00F48844204D14FF6FF700E4981
:1066B00008800CE00D48844203D100200C4908807A
:1066C00005E00C48844202D100200B49088005B047
:1066D00030BD0000000007084E0000200008070839
:1066E000590000200010070850000020001807087B
:1066F0007E00002000200708800000202DE9FF4FC9
:106700008BB08B4690469946199E0020089009F15F
:10671000010258F8221058F82900F9F704FE8246C1
:106720006649F9F738FE07900A960A9EB00000F015
:10673000D5F904464FF0000A12E05046F9F7DBFEA7
:1067400003900799F9F7F5FD049009F1010058F855
:1067500020100498F9F795FD44F82A000AF1010A7F
:10676000B245EADB4FF0FF35554806904FF0000A7E
:1067700022E054F82A100B98F9F7D5FD0190F9F7AB
:10678000F5FE21F00041CDE90201F9F702FF049086
:1067900006990498F9F71AFF01D2504600E02846FE
:1067A000054606990498F9F711FF01D2049800E014
:1067B000069806900AF1010AB245DADB41480590D5
:1067C0000996099EB00000F089F907464FF0000ACB
:1067D00011E05046F9F78FFE3A490390F9F7A9FD09
:1067E000049018985BF820100498F9F74AFD47F8D0
:1067F0002A000AF1010AB245EBDB54F825003249C0
:10680000F9F7EEFE04D248F29010304908804AE0D1
:1068100054F825002E49F9F7E3FE1FD254F825005D
:106820002949F9F7D3FE19D857F82500F9F79EFE44
:1068300021F000410022274BCDE90001F9F7E9FDE5
:10684000CDE90201F9F779FE80B20890089840F48A
:10685000004008901D490898088024E054F825005D
:106860001D49F9F7BDFE10D854F825001849F9F76D
:10687000ADFE0AD857F825001049F9F75AFD8246AF
:10688000F9F747FE114908800DE054F82500124938
:10689000F9F79CFE04D240F21A400C49088002E04D
:1068A00000200A49088000200890384600F016F8B9
:1068B000204600F013F80FB0BDE8F08F0000204133
:1068C00000007A44CDCCCC3DB57DAA43180500200C
:1068D000E9F70242000024408104153F10B500286A
:1068E00021D0114B0022001F196803E0814203D818
:1068F0000A4649680029F9D152B11368841A9C42AA
:1069000004D1006818441060104602E0506000E0B6
:10691000186039B102680B1A934203D10B681A440C
:1069200002604968416010BD080600202DE9FC475F
:1069300081460C461546AFB226462E482E490860C1
:1069400007F50060C11700EB5151C9122B4A1180A5
:106950004FF400612A48F9F782FC2AA103C9CDE966
:1069600000010120294908603CE001221146284825
:10697000FBF788FC0120FBF7EDF9002201212448F8
:10698000FBF780FC4FF4006231461D48FAF7A8F986
:106990004FF48062184801681948FAF7B7F9502097
:1069A000FFF755FE4FF400611548F9F758FC1748FA
:1069B0006A4618A103681948FFF7B2FB80461FFA20
:1069C00088F216491648FDF72FF806F500660A48C2
:1069D000006800F50060084908600C480068401C29
:1069E0000A49086009480068044909888842BCDDF2
:1069F000BDE8FC8700000408400000203C000020A7
:106A00000020002061636B3D000000004400002076
:106A1000000C0140257325640D0A0000843200201B
:106A200030470020FBF746FCFEF7CCFEFDF764FD87
:106A3000FDF7FAFCFDF720FEFDF7B0FCFDF7E4FDE5
:106A4000FDF736FE1948FCF797FAF9F747FF1848A3
:106A500000F070FE174800F009FE174800F0CAFB6E
:106A600013480E3000F038FE144800F0BFFB044617
:106A700000F0B0FD124800F0B9FB044600F0E0FD64
:106A8000FEF764FD4FF480620E490F48FCF754FF97
:106A90000D480068C06840F010000B490968C860E4
:106AA000FDF7ECFC00F05CF800BFFEE7B80F00203B
:106AB0007AF00708004807080000070800080708E0
:106AC00000100708843600203047002001460020CF
:106AD000842901D0CA1C104470470000F0B50B3067
:106AE000154D20F007010024144A0FE003688B4283
:106AF0000BD38B4205D95E1A43184768C3E9006778
:106B000000E04368136002C004E0021D1068002822
:106B1000ECD12046002802D1286808B10020F0BD41
:106B2000064A07481060074A121A22F00702C0E915
:106B3000002401202860D7E70C060020080600206A
:106B4000EC550020E857002070B5044625460DB1ED
:106B5000294600E00121084600F008FF002070BD32
:106B600010B500F031FF002010BD7FB504460D4682
:106B7000606998B1A06988B1B4F90800FFF7A6FF71
:106B80000646D4E90510CDE9006102902B46226942
:106B9000D4E9001001F06CF8039013E0B4F9080098
:106BA000FFF794FF064603A8CDE90060238A9AB256
:106BB0002B46D4E9001001F029F8012802D000206A
:106BC00004B070BD0398FBE72DE9F04105460E4681
:106BD0001C4807681C480068001D00F0CBFD50B938
:106BE0001948006890F82C1001208840174909685E
:106BF000814316480160681C38B936B112480168F3
:106C0000091D134800F000FE1AE07C190E480068C8
:106C10004460BC4207D20C480168091D0D48006859
:106C200000F0D8FD0CE008480168091D0A4800681A
:106C300000F0D0FD09480068844201D20748046092
:106C4000BDE8F081BC050020A8050020C00500209B
:106C5000D4490020B0050020AC050020D805002054
:106C600010B5044600F0DCFD23480068401C2249B2
:106C700008602248006840B920480460084600685F
:106C800001280DD100F03AF90AE01D48006838B932
:106C90001A480068C06AE16A884201D8174804604F
:106CA00018480068401C1749086094F82C1001200F
:106CB000884015490968084313490860E16A01EBF7
:106CC0008101124A02EB8100211D00F09DFD00F0C0
:106CD000D1FD0B48006868B108480068C06AE16AE5
:106CE000884207D24FF0805009490860BFF34F8FA8
:106CF000BFF36F8F10BD0000B8050020A80500206D
:106D0000C4050020D4050020C0050020F84800205C
:106D100004ED00E010B516E000F082FD0C48C068FC
:106D2000C468201D00F026FD0A480068401E09497D
:106D3000086009480068401E0749086000F09AFD95
:106D4000204600F00BF8044800680028E4D110BD8C
:106D5000C0490020B8050020B405002010B5044645
:106D600094F8510030B9206B00F0A2FD204600F0ED
:106D70009FFD1AE094F85100012803D1204600F04D
:106D800097FD12E094F85100022801D1012000E0A3
:106D9000002050B900BF502080F31188BFF34F8FFF
:106DA000BFF36F8F00BF00BFFEE710BD30B54FF4DB
:106DB0004063174800F007042CB1C01D20F0070005
:106DC000134C041B1B1B0246124C22600024114D65
:106DD0006C60D018083820F007000F4C20600024A9
:106DE0000D4D2D686C600C4D2D682C601146441AB9
:106DF0004C60094C24680C60084D4C682C60084DB0
:106E00004C682C604FF00044064D2C6030BD0000F3
:106E1000E8490020E4050020EC050020F4050020EE
:106E2000F0050020F805002000BFFFF773FF0648BB
:106E300000680128F9D94FF0805004490860BFF379
:106E40004F8FBFF36F8FF0E7F848002004ED00E0AC
:106E50002DE9FF5F81460F469246DDE90E6B109CDF
:106E6000AAF10100216B01EB800828F0070808F067
:106E7000070008B9012000E0002050B900BF5020F1
:106E800080F31188BFF34F8FBFF36F8F00BF00BF38
:106E9000FEE7002507E0795D04F134004155785D97
:106EA00000B902E06D1C102DF5D300BF0021432076
:106EB0000155072E00D30626E66266640020A06412
:106EC000201D00F084FC04F1180000F080FC246117
:106ED000C6F10700A06164620020E06484F85000FD
:106EE00049464046039A00F049F92060BBF1000F83
:106EF00001D0CBF80040BDE8FF9F000010B5002492
:106F000007E004EB84010F4A02EB810000F052FC21
:106F1000641C072CF5D30C4800F04CFC0B4800F027
:106F200049FC0B4800F046FC0A4800F043FC0A48C4
:106F300000F040FC0448094908600448084908601A
:106F400010BD0000F8480020844900209849002026
:106F5000AC490020C0490020D4490020AC050020E5
:106F6000B005002010B50146164800E0006803682F
:106F70008B42FBD30246436813448B4204D14368DF
:106F80004C682344436001460A464B681344046836
:106F9000A34211D10C4C03682468A34208D04B686B
:106FA0000468646823444B6003681B680B6005E059
:106FB000054B1B680B6001E003680B60884200D042
:106FC000016010BDE4050020EC0500200A490968B5
:106FD000096809B9012100E0002121B14FF0FF311A
:106FE000064A116006E004490968C968C868034A8E
:106FF0004168116070470000AC050020D8050020F2
:107000000E480068401C08B9012000E0002050B97B
:1070100000BF502080F31188BFF34F8FBFF36F8FF5
:1070200000BF00BFFEE700BF502080F31188BFF310
:107030004F8FBFF36F8F00BF00BFFEE7FC0500203E
:107040002DE9F04104464FF0000800F015FD4648D8
:10705000006808B9FFF7AAFE4448006820400028ED
:107060006BD1D4B1083404F00700B0B104F00700CC
:10707000C0F10800044404F0070008B9012000E052
:10708000002050B900BF502080F31188BFF34F8F0C
:10709000BFF36F8F00BF00BFFEE7002C4DD0344818
:1070A0000068844249D8334E3046056801E02E46D8
:1070B0002D686868A04202D228680028F7D12A48C3
:1070C0000068854239D0306800F1080828683060CF
:1070D0006868001B102819D92F1907F0070008B994
:1070E000012000E0002050B900BF502080F311883B
:1070F000BFF34F8FBFF36F8F00BF00BFFEE768681D
:10710000001B78606C603846FFF72CFF18496868F0
:107110000968081A1649086008460068164909688F
:10712000884203D212480068134908600F49686812
:107130000968084368600020286000F099FE08F0A4
:10714000070008B9012000E0002050B900BF50201E
:1071500080F31188BFF34F8FBFF36F8F00BF00BF65
:10716000FEE74046BDE8F081EC050020F805002070
:10717000F0050020E4050020F4050020001F4FF07A
:1071800080730360001F21F001030360001F034BA5
:107190000360143802602038704700000170000856
:1071A00010B50548FCF792F84FF480620349024895
:1071B000FCF7C2FB10BD00003047002084360020E1
:1071C00002460948006838B1002002E00B5C135405
:1071D000401C0528FADB06E0002002E00B5C13549B
:1071E000401C0428FADB70472C0000200146088868
:1071F0007047000010B504462046FFF7F7FF03462E
:107200004FF6FF70834204D103480088024908808A
:1072100001E00148038010BD4E0000202DE9FE4F23
:1072200006460F4690461D46DDE90C9A0E9C00204E
:10723000009001900290F0B28DF800008DF801707E
:107240008DF8028028128DF80300E8B28DF8040052
:107250004FEA29208DF8050009F0FF008DF806009F
:107260004FEA2A208DF807000AF0FF008DF8080089
:10727000A01EC1B26846FFF759F983460BF0FF0123
:10728000A01E0DF800104FEA2B21601E0DF8001013
:10729000631EA2B269460448FCF76DFBFFF77EF956
:1072A000FFF77EFFBDE8FE8F304700202DE9F04F4D
:1072B00085B006460F4690461D46DDE90FABDDF86A
:1072C0003890119C00200190029003900490F0B23D
:1072D0008DF804008DF805708DF8068028128DF861
:1072E0000700E8B28DF808004FEA29208DF8090060
:1072F00009F0FF008DF80A004FEA2A208DF80B00F4
:107300000AF0FF008DF80C004FEA2B208DF80D00DD
:107310000BF0FF008DF80E00A01EC1B201A8FFF710
:1073200005F900900098C1B2A01E01AA115400985E
:107330000112601E1154631EA2B201A90448FCF799
:107340001AFBFFF72BF9FFF72BFF05B0BDE8F08F15
:10735000304700202DE9F04F85B006460F46904695
:107360001D46DDE911B4DDE90E9A0020019002907E
:1073700003900490F0B28DF804008DF805708DF83C
:10738000068028128DF80700E8B28DF808004FEA51
:1073900029208DF8090009F0FF008DF80A004FEA56
:1073A0002A208DF80B000AF0FF008DF80C001098D1
:1073B00000128DF80D001098C0B28DF80E004FEA43
:1073C0002B208DF80F000BF0FF008DF81000A01E91
:1073D000C1B201A8FFF7AAF800900098C1B2A01EA0
:1073E00001AA115400980112601E1154631EA2B22A
:1073F00001A90548FCF7BFFAFFF7D0F8FFF7D0FE68
:1074000005B0BDE8F08F0000304700202DE9FC47B3
:1074100006460F4690461D460A9C002000900190AB
:10742000F0B28DF800008DF801708DF802802812FE
:107430008DF80300E8B28DF80400A01EC1B26846C2
:10744000FFF774F8814609F0FF01A01E0DF8001047
:107450004FEA2921601E0DF80010A2B223466946AA
:107460000448FCF788FAFFF799F8FFF799FEBDE8A2
:10747000FC870000304700202DE9FC410746884684
:1074800014461D46002000900190F8B28DF80000CF
:107490008DF8018020128DF80200E0B28DF8030013
:1074A00028128DF80400E8B28DF805000621684620
:1074B000FFF73CF80646F0B28DF8060030128DF862
:1074C00007000723082269460448FCF754FAFFF72F
:1074D00065F8FFF765FEBDE8FC810000304700203D
:1074E0002DE9FE4F06460F4690461D46DDE90C94F9
:1074F0000020009001900290F0B28DF800008DF80D
:1075000001708DF8028028128DF80300E8B28DF822
:1075100004004FEA29208DF8050009F0FF008DF8DE
:107520000600A01EC1B26846FFF700F882460AF0C6
:10753000FF01A01E0DF800104FEA2A21601E0DF871
:107540000010631EA2B269460448FCF714FAFFF764
:1075500025F8FFF725FEBDE8FE8F0000304700202C
:107560002DE9FE4306460F4614461D46DDF82890D9
:107570000020009001900290F0B28DF800008DF88C
:10758000017020128DF80200E0B28DF8030028127D
:107590008DF80400E8B28DF805008DF806900721FB
:1075A0006846FEF7C3FF804608F0FF008DF807002D
:1075B0004FEA28208DF8080009231A466946044836
:1075C000FCF7D9F9FEF7EAFFFFF7EAFDBDE8FE8315
:1075D0003047002010B504464FF6FF70844214D1A6
:1075E000002208211548FAF74DFE00221021134809
:1075F000FAF748FE002220211048FAF743FE002245
:1076000040210E48FAF73EFE17E004F0010208217F
:107610000A48FAF737FEC4F3400210210748FAF788
:1076200031FEC4F3800220210448FAF72BFEC4F394
:10763000C00240210148FAF725FE10BD000C0140B0
:1076400010B50446072C04DC074951F82400FEF766
:1076500089FF4FF6FF70844201D0032C03D14FF411
:107660001650FEF77FFF10BD3805002010B5044608
:10767000022221461648F9F733FB00200FE0144997
:1076800031F810104FF47F4202EA0121104A32F81B
:10769000102041EA12210E4A22F81010401C012845
:1076A000EDDB0B4800884FF6FF71884203D10020C4
:1076B000084908600BE0064800884FF47F4101EA62
:1076C00000200349098840EA11200249086010BDE2
:1076D000300500202000002038B504460822124959
:1076E0001248F9F7FDFA00200FE0104931F81010A8
:1076F0004FF47F4202EA01210C4A32F8102041EA9D
:1077000012210A4A22F81010401C0428EDDB6946B9
:107710000648FEF75DFF0098401C00B938BD0449DB
:107720000098086000BFF9E788F007080200002011
:107730005400002010B5044610220C490C48F9F7FB
:10774000CFFA00200FE00A4931F810104FF47F42C1
:1077500002EA0121064A32F8102041EA1221044AC5
:1077600022F81010401C0828EDDB10BD005007085F
:107770007206002001460A69D1E901309860D1E91A
:10778000010358605068884201D188685060002029
:1077900008611068401E106010687047034B03605A
:1077A000034B0B60802313607047000030300020D3
:1077B0008430002000F1080141604FF0FF3181600A
:1077C00000F10801C16001610021016070470021E2
:1077D0000161704710B502460B685C1C0CB910695A
:1077E00007E002F1080000E04068446824689C4219
:1077F000FAD944684C604C68A160886041600A61B5
:107800001468641C146010BD42684A6093688B6001
:10781000936859609160086103685B1C036070475E
:1078200000BF502080F31188BFF34F8FBFF36F8FDD
:1078300000BF0E480068401C0C49086008460068FC
:10784000012812D10A480068C0B208B9012000E03E
:10785000002050B900BF502080F31188BFF34F8F34
:10786000BFF36F8F00BF00BFFEE77047FC0500202D
:1078700004ED00E00D48006850B900BF502080F3CF
:107880001188BFF34F8FBFF36F8F00BF00BFFEE7BC
:1078900006480068401E054908600846006820B98F
:1078A000002080F3118800BF00BF7047FC05002056
:1078B00070B506463546002E3FD0083D2C461F4980
:1078C00060680968084008B1012000E0002050B954
:1078D00000BF502080F31188BFF34F8FBFF36F8F2D
:1078E00000BF00BFFEE7206808B9012000E00020CB
:1078F00050B900BF502080F31188BFF34F8FBFF302
:107900006F8F00BF00BFFEE70C4960680968084040
:1079100098B1206888B9094960680968884360603F
:1079200000F0AAF80649606809680844044908603C
:107930002046FFF717FB00F09BFA70BDF80500200A
:10794000F005002000204FF0E02108618861064822
:1079500000684FF47A71B0FBF1F0401E4FF0E02167
:107960004861072008617047A405002070B50446EF
:107970000025D4B11248006808B9012000E00020B9
:1079800050B900BF502080F31188BFF34F8FBFF371
:107990006F8F00BF00BFFEE700F06EF800212046A9
:1079A000FFF712F900F064FA05463DB94FF0805038
:1079B00004490860BFF34F8FBFF36F8F70BD0000A5
:1079C000E005002004ED00E010B586B00020059031
:1079D000049003AA04A905A8FFF7E0FE0022DDE950
:1079E00004101346CDE9002102901CA11D48039A02
:1079F00000F03EF91C4908600846006808B10124FF
:107A000000E00024012C15D100BF502080F3118824
:107A1000BFF34F8FBFF36F8F00BF4FF0FF3013499D
:107A2000086001201249086000201249086000F037
:107A300071F810E0601C08B1012000E0002050B98E
:107A400000BF502080F31188BFF34F8FBFF36F8FBB
:107A500000BF00BFFEE706B010BD000049444C4522
:107A600000000000296E0008DC050020D805002079
:107A7000C4050020BC05002002480068401C0149E4
:107A800008607047E00500201D48006818B101201B
:107A90001C49086032E000201A4908601A48006852
:107AA000B0FA80F0C0F11F0101EB8100174A52F8D3
:107AB000200008B1012000E0002050B900BF502094
:107AC00080F31188BFF34F8FBFF36F8F00BF00BFEC
:107AD000FEE701EB81020D4B03EB82004268526826
:107AE000426000F108024368934202D14268526842
:107AF00042604268D268064B1A6000BF70470000BF
:107B0000E0050020CC050020C0050020F84800203A
:107B1000A80500201CB53849084600780190FF20D0
:107B20000A4610700846007800909DF8000000F0AA
:107B3000F0009DF80020904201D1012000E00020DB
:107B400050B900BF502080F31188BFF34F8FBFF3AF
:107B50006F8F00BF00BFFEE79DF8000000F05000EF
:107B6000264A10700720264A106009E02448006861
:107B7000401E234A10609DF800004006000E009051
:107B80009DF8000000F080008028EFD01C480068BD
:107B9000C0F10700042801D1012000E0002050B905
:107BA00000BF502080F31188BFF34F8FBFF36F8F5A
:107BB00000BF00BFFEE7124800680002104A1060D4
:107BC0001046008800F4E06010600B4A01981070C5
:107BD0000C48006840F470000A49086008460068D4
:107BE00040F070400860FFF7ADFE002006490860D5
:107BF000F8F7C0FA00201CBD00E400E000060020F9
:107C00000406002020ED00E0FC0500202DE9FF4FD8
:107C100085B0804689461746DDE912ABB800FFF70C
:107C20000FFA064656B15420FFF70AFA04460CB183
:107C3000266304E03046FFF73BFE00E000248CB1F1
:107C4000002084F85100CDE900ABCDE902403A466E
:107C500049464046089BFFF7FBF82046FFF700F82F
:107C6000012501E04FF0FF35284609B0BDE8F08F4F
:107C70002DE9F04F85B00746884691469A46DDE9E2
:107C80000EB6109C0EB1012000E0002050B900BFDC
:107C9000502080F31188BFF34F8FBFF36F8F00BF69
:107CA00000BFFEE70CB1012000E0002050B900BF8A
:107CB000502080F31188BFF34F8FBFF36F8F00BF49
:107CC00000BFFEE7542003900398542801D10120FF
:107CD00000E0002050B900BF502080F31188BFF3AE
:107CE0004F8FBFF36F8F00BF00BFFEE7B4B1AEB1DF
:107CF00025462C462E63022085F85100002004A959
:107D000053464A46CDE900B1CDE9025041463846D6
:107D1000FFF79EF82846FEF7A3FF01E0002004903D
:107D2000049805B0BDE8F08F2DE9F0414FF0000850
:107D300044480068002877D143480068451C424801
:107D4000056015BB41480068006808B9012000E0E3
:107D5000002050B900BF502080F31188BFF34F8F2F
:107D6000BFF36F8F00BF00BFFEE738480768384891
:107D70000068364908603648076036480068401C8D
:107D800034490860FFF722F900BF33480068854294
:107D90003CD300BF2D480068006808B9012000E00E
:107DA000002020B14FF0FF302B4908602DE027481C
:107DB0000068C068C4686668B54202D2264806609A
:107DC00023E0201DFFF7D6FCA06A18B104F11800CB
:107DD000FFF7D0FC94F82C10012088401F49096857
:107DE00008431E490860E16A01EB81011C4A02EB6D
:107DF0008100211DFFF708FD1A49E06A0968C96A78
:107E00008842C7D34FF00108C4E700BF1548006897
:107E1000C06A00EB8000124951F82000012801D906
:107E20004FF0010805E0FFE70F480068401C0E49CD
:107E300008600E48006808B14FF001084046BDE8F0
:107E4000F0810000E0050020BC050020AC0500200A
:107E5000B0050020D0050020D8050020C005002076
:107E6000F8480020A8050020C8050020CC05002007
:107E700070B5002400263648006850B900BF502075
:107E800080F31188BFF34F8FBFF36F8F00BF00BF28
:107E9000FEE7FFF7C5FC2E480068401E2C4908602D
:107EA0000846006800284FD12A48006800284BD0B7
:107EB00024E02948C068C46804F11800FFF75AFCA0
:107EC000201DFFF757FC94F82C100120884023490F
:107ED0000968084321490860E16A01EB8101204AF1
:107EE00002EB8100211DFFF78FFC1E49E06A096843
:107EF000C96A884202D301201B49086016480068FD
:107F000008B9012000E000200028D2D00CB1FFF712
:107F10005DF81648056865B100BFFFF705FF10B1B1
:107F20000120114908606D1E002DF6D100200F4977
:107F300008600D48006838B1012630070C49086018
:107F4000BFF34F8FBFF36F8FFFF794FC304670BDC8
:107F5000E0050020B8050020AC490020C005002045
:107F6000F8480020A8050020CC050020C805002006
:107F700004ED00E00008014001000000000801409D
:107F80000200000000080140040000000008014059
:107F90000800000000080140100000000008014037
:107FA00020000000000801404000000000080140DF
:107FB00080000000848000082957000803000000AA
:107FC0000000000080000000000000000000000031
:107FD00060800008ED54000803000000000000006D
:107FE0008000000000000000000000006C8000081D
:107FF0003955000803000000000000008000000068
:1080000000000000000000007880000843550008D0
:1080100003000000000000008000000000000000DD
:108020000000000002030405060708090A0B0C0DF6
:108030000E0F1010010202030405060708090A0BBF
:108040000C0D0E0F101001020000000000000000D7
:1080500001020304060708090000000001020304EE
:108060006D795461736B3032000000006D7954619A
:10807000736B3033000000006D795461736B3034E2
:10808000000000006961705461736B00AC800008EF
:1080900000000020100600008A070008E0840008A5
:1080A00010060020D8550000D0610008011E032EE4
:1080B000060862C1042E0708232320C21A1C041AD2
:1080C00018041A14041A10041A0C041A08041A04C6
:1080D000041119041AF85D1AF0041AE8041AE004ED
:1080E0001AD8041AD0041AC8041AC0041AB8041AF8
:1080F000B0041AA8041AA0041A98041A90041A8842
:10810000041A80041A70041A60041A50041A4004F5
:108110001A30041A20042A10B529541AC048190428
:108120001AA0041A80041A400411290C62BF33807B
:108130003F1A400319041A80041AA0041AC0041A32
:10814000E004111A414819041A20041A30041A4094
:10815000041A50041A60041A70041A80041A88045D
:108160001A90041A98041AA0041AA8041AB0041A3F
:10817000B8041AC0041AC8041AD0041AD8041AE0A1
:10818000041AE8041AF0041AF8041122421A04042A
:108190001A08041A0C041A10041A14041A18041ADF
:1081A0001C041A20041A24041A28041A2C041A3055
:1081B000041A34041A38041A3C041A40041A4404F9
:1081C0001A48041A4C041A50041A54041A58041A6F
:1081D0005C041A60041A64041A68041A6C041A70A5
:1081E000041A74041A78041A7C041A80041A82048B
:1081F0001A84041A86041A88041A8A041A8C041A27
:108200008E041A90041A92041A94041A96041A9866
:10821000041A9A041A9C041A9E041AA0041AA204AE
:108220001AA4041AA6041AA8041AAA041AAC041A56
:10823000AE041AB0041AB2041AB4041AB6041AB876
:10824000041ABA041ABC041ABE041AC0041AC204DE
:108250001AC4041AC6041AC8041ACA041ACC041A86
:10826000CE041AD00400FF00D242CC76AA43487054
:108270009F43EB32954324AF8B43A5D68243A1386D
:1082800075433EE8654318A65743D95D4A43E0FC71
:108290003D4313723243A5AD274313A11D43FA3E5C
:1082A00014430F7B0B43EF4903434142F742FAED7E
:1082B000E8421F85DB423FF7CE421835C3427D308E
:1082C000B8426ADCAD42E72CA442A1169B42428F21
:1082D0009242438D8A42A107834271EC774282A287
:1082E0006A4254235E42B16152424E514742B5E662
:1082F0003C423F17334217D92942EB2221423DEC41
:1083000018420E2D114201DE0942E9F7024210E93E
:10831000F841719BEC41B3FBE0412EFFD541439CFA
:10832000CB4186C9C141917EB84133B3AF41D95FDA
:10833000A741BF7D9F41F00598417CF29041713D7E
:108340008A41B1E1834168B37B41F2417041666685
:10835000654159175B41D34D51410C0248410E2DE7
:108360003F414BC8364120099FCD2E414C37274114
:108370001015204168221941029A12417C610C417A
:108380008E750641B7D118F9418FE4F6401EA7EC6F
:10839000408FE4E2405396D940AEB6D040143FC877
:1083A000406B2BC040C976B840A01AB1407B14AADC
:1083B000409E5EA340C3F59C40D0D596407FFB9085
:1083C00040B7628B40D50986401CEB80401B0D787E
:1083D000407DAE6E4017B76540A3235D40EEEB5481
:1083E00040B30C4D404D8445408C4A3E40705F3751
:1083F000400EBE30407C612A4017482440986E1ED3
:10840000405BD318407671134045470E40835109B5
:10841000408A8E044072F9FF3F9031F73F27C2EE49
:108420003FA9A4E63F5DDCDE3F705FD73FE02DD083
:108430003F2041C93F3199C23FCA32BC3FA60AB66C
:108440003F7E1DB03F0A68AA3F4BEAA43FF9A09FB8
:108450003FCE889A3FCBA1953FA7E8903F1D5A8C0D
:108460003F72F9873F1AC0833F9B557F3FA77977BB
:108470003F57EC6F3F029A683FC58F613F83C05AF8
:1084800048003310543F0DE04D3FBEC1473FDCD79D
:10849000413FF6283C3FF0A7363FCA54313F1136E2
:1084A0002C3FAB3E273F2575223FF2D21D3F10588F
:1084B000193F8104153F5AFF01C123B0042360090D
:1084C00023C012338025324B329632E113C20102AF
:1084D000438032104201035524F41AAA010110000E
:0400000508000131BD
:00000001FF
